:0200000480007A
:10000000B72F0000938F0F8073900F3015A8130047
:100010000000130000001300000013000000130094
:100020000000130000001300000013000000130084
:100030000000130000001300000013000000010086
:10004000970200009382020C73905230814001416C
:100050008141014281420143814301448144014580
:100060008145014681460147814701488148014950
:100070008149014A814A014B814B014C814C014D20
:10008000814D014E814E014F814F971102009381A6
:1000900021D5170502001305E556979503009385B2
:1000A000257E01461122170502001305E54A970532
:1000B00002009385A5520146C52817A50300130524
:1000C000657C97B503009385A57B37B6ABAB13066C
:1000D000B6BAD92817B103001301C17AEF6060796D
:1000E000860293D21200F512638802008242110147
:1000F0006F00001073002030824211017300203025
:10010000711116C0F3222034E3CC02FC82421101AB
:10011000130141F806C20AC40EC612C816CA1ACC88
:100120001ECE22D026D22AD42ED632D836DA3ADCC7
:100130003EDEC2C0C6C2CAC4CEC6D2C8D6CADACC97
:10014000DECEE2D0E6D2EAD4EED6F2D8F6DAFADCA7
:10015000FEDE73252034F32510340A8601A07310C7
:10016000153492402241B2414242D2426243F243AC
:10017000025492542255B2554256D2566257F25703
:10018000064896482649B649464AD64A664BF64B33
:10019000065C965C265DB65D465ED65E665FF65F83
:1001A0001301C1077300203010C16374B50011053D
:1001B000E5BF828000000000000000000000000099
:1001C000000000000000000000000000000000002F
:1001D000000000000000000000000000000000001F
:1001E000000000000000000000000000000000000F
:1001F000197106C00AC20EC412C616C81ACA1ECC8D
:1002000022CE26D02AD22ED432D636D83ADA3EDCC6
:1002100042DEC6C0CAC2CEC4D2C6D6C8DACADECC96
:10022000E2CEE6D0EAD2EED4F2D6F6D8FADAFEDCA6
:100230009702020083A2823523A02200F322103409
:1002400096DEEF00002B170102000321213402414A
:10025000F65273901234B72200009382028873A082
:10026000023082403242C2425243E24372448254DC
:100270001255A2553256C2565257E2577258864806
:100280001649A649364AC64A564BE64B764C865C1A
:10029000165DA65D365EC65E565FE65F0961730059
:1002A0002030970202009382E23523A0120023A29D
:1002B000220023A4320023A6420023A8520023AA2E
:1002C000620023AC720023AE820023A0920223A21C
:1002D000A20223A4B20223A6C20223A8D20223AA06
:1002E000E20223ACF20223AE020323A0120523A2F2
:1002F000220523A4320523A6420523A8520523AADA
:10030000620523AC720523AE820523A0920723A2C7
:10031000A20723A4B20723A6C20723A8D20723AAB1
:10032000E20723ACF207EF40702717010200032118
:10033000E1250241F65273901234B72200009382F5
:10034000028873A0023082403242C2425243E243EA
:10035000724482541255A2553256C2565257E25731
:10036000725886481649A649364AC64A564BE64B45
:10037000764C865C165DA65D365EC65E565FE65FB1
:10038000096173002030970202009382A22783A0A4
:10039000020003A1420083A1820003A2C20083A243
:1003A000020103A3420183A3820103A4C20183A427
:1003B000020203A5420283A5820203A6C20283A60B
:1003C000020303A7420383A7820303A8C20383A8EF
:1003D000020403A9420483A9820403AAC20483AAD3
:1003E000020503AB420583AB820503ACC20583ACB7
:1003F000020603AD420683AD820603AEC20683AE9B
:10040000020703AFC20983AF820782807370043092
:10041000197106C00AC20EC412C616C81ACA1ECC6A
:1004200022CE26D02AD22ED432D636D83ADA3EDCA4
:1004300042DEC6C0CAC2CEC4D2C6D6C8DACADECC74
:10044000E2CEE6D0EAD2EED4F2D6F6D8FADAFEDC84
:100450009702020083A2821323A0220086DEEF20EF
:10046000602E17010200032161120241F6527390BF
:100470001234B72200009382028873A002308240B7
:100480003242C2425243E243724482541255A25550
:100490003256C2565257E257725886481649A649F4
:1004A000364AC64A564BE64B764C865C165DA65DD0
:1004B000365EC65E565FE65F09617300203073707A
:1004C000043001A07310453082807325403073F0F2
:1004D00043308280970700009387A7FE232EB5FE46
:1004E0002322C5FA232635F82320F5F8130505F84D
:1004F0008280411106C6EF409007EF10900A01E597
:10050000B24041018280B24041016F20A023930795
:1005100085007D575CC118C55CC51CC9232005003A
:1005200082802328050082805C41DCC1984798C501
:1005300098474CC38CC788C91C4185071CC1828061
:100540009041FD57130785006314F60039A83E87D4
:100550005C439443E37DD6FEDCC18CC798C54CC395
:1005600088C91C4185071CC1828018495C43EDB7CE
:10057000584114451C4914C71845544154C3D84325
:100580006314A7001845D8C32328050088437D15A8
:1005900088C382803041AE8701CE4C455841B29528
:1005A0004CC563E4E5000C414CC53E856F30B0207E
:1005B0008280411122C406C62A8426C2EF2030124E
:1005C0003C44635BF0025C5085CB9304440209A871
:1005D0003C44FD173CC43C446350F0025C5089CF5E
:1005E0002685EF2040586DD5EF2020783C44FD173C
:1005F0003CC43C44E344F0FEFD573CC4EF20701083
:10060000EF20F00D7C40635BF0021C4885CB930427
:10061000040109A87C40FD177CC07C406350F002B7
:100620001C4889CF2685EF2000546DD5EF20E0735C
:100630007C40FD177CC07C40E344F0FEFD577CC04D
:100640002244B240924441016F20B00B29CD0111E8
:1006500022CC2A8406CE26CA4AC84EC62E89EF204E
:10066000100824404C5C832904002685EF600002BA
:100670007D57232C0402B3079540CE974E9578C042
:1006800048C0232434015CC438C4631109021C48E7
:100690008DE7EF201007F2406244D2444249B2494C
:1006A0000545056182807370043001A013050401C3
:1006B000B93D13054402A13DE9BF13050401EF2034
:1006C000804A8547E317F5FC9133E1B701E5737084
:1006D000043001A0011126CA4AC84EC606CE22CC5B
:1006E000AA842E89B289A5C9EF50507A1305550501
:1006F000EF3020742A8435C5930745051CC144DCBE
:1007000023202405EF20A07D24404C5C0329040015
:100710002685EF50B077FD56232C0402B307954091
:100720003307A900CA9774C058C05CC434C4130509
:10073000040123242401E13B13054402C93BEF20BB
:10074000407C230834052285F2406244D244424969
:10075000B2490561828013054005EF30806D2A841F
:1007600001E57370043001A000C051BF01E5737052
:10077000043001A06375B5007370043001A041110D
:1007800022C409462E84814506C6893711C500DD7D
:10079000B2402244410182807370043001A05D7137
:1007A00086C6A2C4A6C2CAC04EDE52DC56DA5AD8E9
:1007B0005ED632C6630A051C6382051C89476399AD
:1007C000F600585D85476305F7007370043001A09B
:1007D0003689AE842A84EF20C05B11E5B24781C719
:1007E0007370043001A0EF20806F185C5C5C014BDB
:1007F000894BFD59130A0401930A44026365F70CFF
:1008000063077919B2476381072463150B00280831
:10081000EF208048EF20E06EEF10604FEF20206C5B
:100820007C4063943701232204043C4463943701E1
:1008300023240404EF20E06C6C002808EF20E0473C
:10084000631E051EEF20A069185C5C5C630CF70A50
:10085000EF20206BEF20A0683C44634FF00039A8E4
:100860005685EF20403019C1EF2020503C44FD1741
:100870003CC43C446354F0005C50FDF32324340535
:10088000EF202068EF20A0657C40634FF00039A87E
:100890005285EF20402D19C1EF20204D7C40FD17DF
:1008A0007CC07C406354F0001C48FDF323223405D7
:1008B000EF202065EF10A06A054BEF204062185C26
:1008C0005C5CE37FF7F230406305060C631F09129E
:1008D0000844A685EF30206E1C4434405840B6973B
:1008E0001CC463EAE70A1C5C14405850850714C412
:1008F0001CDC5DC713054402EF20E0268547631129
:10090000F50AC9A8EF20E05FB2455285EF206007E5
:10091000EF20E05C3C44634FF00039A85685EF209F
:10092000802419C1EF2060443C44FD173CC43C4482
:100930006354F0005C50FDF323243405EF20605C29
:10094000EF20E0597C40634FF00039A85285EF203A
:10095000802119C1EF2060417C40FD177CC07C40A4
:100960006354F0001C48FDF323223405EF20605946
:10097000EF10E05E31F1593C054B81B73C41E38F0C
:1009800007E27370043001A07370043001A030409E
:1009900021E61C4085C71C5C585085071CDC39FBD0
:1009A000EF2020560545B640264496440649F259A4
:1009B000625AD25A425BB25B616182804840EF204A
:1009C00060491C5C58502322040085071CDCE3139B
:1009D00007F279D5253CE9B74844A685EF30A05DFC
:1009E0003C4058441440B307F0403E9758C4637CE1
:1009F000D7025840BA975CC409475C506306E902C5
:100A0000185C050718DCC9DFF5B54844A685EF304A
:100A1000805A3C4058441440B307F0403E9758C4B5
:100A2000E37CD7FCF9B75C50185C79DB185C7D1768
:100A300018DC185C050718DCA5D76DBD2285953E2E
:100A4000EF10E051014585B7EF20A04B0145A1BF54
:100A5000411126C2AA841305400522C406C6EF3000
:100A6000403D2A8415CD232C0502FD577CC1054746
:100A7000410558DC3CC42322040023200400232425
:100A80000400232604002320040423089404413492
:100A900013054402AD3C8146014681452285013360
:100AA0002285B24022449244410182800DC5411109
:100AB00022C426C206C64AC0032945002A84EF2064
:100AC000802C8144630CA900B2402244268502494F
:100AD0009244410182807370043001A05C448544DB
:100AE000FD175CC4F5F381460146814522854539F1
:100AF000E1BF31CDA1C9011122CC26CA4AC852C4D6
:100B000006CE4EC68947B68432892E8A2A846399D6
:100B1000F600585D8547630FF7047370043001A039
:100B20006D32185C5C5CAA896366F70281444E856D
:100B3000513AF240624426854249D244B249224A9F
:100B4000056182803C41C5DB7370043001A0737085
:100B5000043001A0304041E21C40D5CB1C5C7D57E5
:100B600085071CDC3C446387E7083C4485448507D3
:100B70003CC475BF993A185C5C5CAA89636DF70246
:100B8000304079DA4844D285EF30E0423C40584466
:100B90001440B307F0403E9758C46375D7005840DF
:100BA000BA975CC48947E39BF4FA1C5CC5DB1C5C08
:100BB000FD171CDC65B7304045D24844D285EF3084
:100BC000803F3C4058441440B307F0403E9758C41F
:100BD000E367D7FCD9BFDDF40844D285EF30A03DF0
:100BE0001C4434405840B6971CC4E3E9E7F61C4067
:100BF0001CC4ADB75C5085449DDB13054402EF1067
:100C0000907615D5E30509F2232099000DB74840E9
:100C1000EF2040242322040091B721CD3C4181C71D
:100C20007370043001A01C41A1CB011122CC26CA53
:100C30002A844AC84EC606CE2E894138185C5C5CB0
:100C4000AA898144637DF7001C5C7D5785071CDC05
:100C50003C446388E7023C44854485073CC44E8598
:100C60009530F240624426854249D244B24905613A
:100C700082807370043001A05C41C5DB7370043066
:100C800001A05C5099E38544D9BF13054402EF10DD
:100C9000906D75D9E30909FE85472320F900E5B772
:100CA000397106DE22DC26DA4AD84ED652D456D224
:100CB00032C66302051C638A051AB68AAE892A8485
:100CC000EF20200D11E5B24781C77370043001A0F9
:100CD000EF20E0201C5C63920714B247638E070A82
:100CE0002808EF10707BFD5413094402130A040115
:100CF000EF202021EF10A001EF20601E7C406394C4
:100D00009700232204043C446394970023240404A2
:100D1000EF20201F6C002808EF10307A63130518AD
:100D2000EF20E01B1C5CADCFEF20A01DEF20201BAF
:100D30003C44634FF00039A84A85EF10D06219C1D6
:100D4000EF20A0023C44FD173CC43C446354F00037
:100D50005C50FDF324C4EF20C01AEF2040187C4003
:100D6000634FF00039A85285EF10F05F19C1EF1002
:100D7000D07F7C40FD177CC07C406354F0001C4851
:100D8000FDF364C0EF20E017EF10601DEF20201589
:100D90001C5CC1E7B247A9FFEF20A016014555A092
:100DA000EF2020161C40DDC7B2454A85EF10703D8C
:100DB000EF20E0123C44634FF00039A84A85EF1061
:100DC000905A19C1EF10707A3C44FD173CC43C4462
:100DD0006354F0005C50FDF324C4EF208012EF2038
:100DE00000107C40634FF00039A85285EF10B057D7
:100DF00019C1EF1090777C40FD177CC07C40635494
:100E0000F0001C48FDF364C0EF20A00FEF10201588
:100E100031C9EF20C00C1C5CB5DFCE85228544446F
:100E2000EFF04FF7639C0A041C5C1840FD171CDCB4
:100E300001E7EF20801148C01C48A1EFEF20600CB3
:100E40000545F2506254D2544259B259225A925A2C
:100E500021618280EF20A0084840EF109075EF20BC
:100E6000400A99B7EFF08FDA6DB73C41E38707E4AA
:100E70007370043001A07370043001A05C5044C44E
:100E8000D5DF13054402EF10104E4DD9EFF00FD807
:100E900075B713050401EF10104D8547E310F5FAFF
:100EA000F5B72285EFF0EFF0EF10600B014551BF71
:100EB0001DC9411122C44AC006C626C244412E891A
:100EC0002A84EF10506C6383A40281464A868145D0
:100ED0002285F93385476300F502B24022449244EB
:100EE0000249410182807370043001A05C440545D1
:100EF00085075CC4DDB75C4485075CC4F9BF15CDCC
:100F0000ADC9011122CC26CA4AC84EC652C42A8491
:100F100006CE3289AE89EFF04FDB1C5C2A8A814411
:100F200085E35285EFF00FDAF240624426854249AC
:100F3000D244B249224A056182807370043001A014
:100F4000304001CE4C445C40B2954CC463E4F500A3
:100F50000C404CC44E85EF3000061C5C7D57FD17DD
:100F60001CDC7C40638CE7007C40854485077CC0AA
:100F70004DBF3C41D9D77370043001A01C4899E3A0
:100F8000854445B713050401EF10F03D75D9E30919
:100F900009FE85472320F900E5B721C93C41A1CDD1
:100FA000A1CB011122CC26CA4AC852C42A8406CE3B
:100FB0004EC62E8AEFF06FD11C5C2A89814491CBFA
:100FC0008329C400D2852285EFF0CFDC8544232617
:100FD00034014A85EFF00FCFF24062442685424942
:100FE000D244B249224A056182807370043001A064
:100FF0007370043001A0EDDF7370043001A001E5CF
:101000007370043001A0411122C42A8406C6EF1077
:10101000106D005CEF10F06EB24022852244410159
:10102000828001E57370043001A0411106C622C41C
:101030002A84EF10D06A1C5C405C1D8CEF10706C31
:101040002285B24022444101828019C1085D82801C
:101050007370043001A01DCD978703009387877EAE
:10106000D843630CE502D847630CE504D84B63070B
:10107000E504D84F6302E504D853630DE502D85761
:101080006308E502D85B6303E502D85F630EE50001
:101090006F20506C7370043001A001470E07BA979F
:1010A00023A007006F20106B1D47CDBF1947FDB768
:1010B0001547EDB71147DDB70D47CDB70947F9BF64
:1010C0000547E9BF684582806CC5828003450505F8
:1010D000828009C5085D1335150082807370043065
:1010E00001A019C51C5D485D1D8D1335150082805A
:1010F0007370043001A0978703009387A774984307
:1011000005C3984705C7984B05C7984F05C798531F
:1011100005C7985705C7985B15C7985F15C38280A8
:1011200001470E07BA978CC3C8C382800547D5BF55
:101130000947C5BF0D47F5B71147E5B71547D5B7FF
:101140001D47C5B71947F1BF978703009387876F7E
:10115000D8436308E502D847630BE502D84B630A1E
:10116000E502D84F6309E502D8536308E502D85772
:101170006307E502D85B6308E502D85F6303A70253
:10118000828001470E07BA9723A007008280054797
:10119000D5BF0947C5BF0D47F5B71147E5B7154797
:1011A000D5B71D47C5B71947F1BF411122C426C2A3
:1011B0004AC02A8406C6AE843289EF105052784065
:1011C000FD576314F700232204043844FD576314C9
:1011D000F70023240404EF10D0521C5C99E74A86E0
:1011E000A68513054402EF10D00CEF10504F3C447D
:1011F000635BF0025C5085CB9304440209A83C4435
:10120000FD173CC43C446350F0025C5089CF2685F6
:10121000EF1070156DD5EF1050353C44FD173CC4F0
:101220003C44E344F0FEFD573CC4EF10904DEF10FA
:10123000104B7C40635BF0021C4885CB9304040197
:1012400009A87C40FD177CC07C406350F0021C481C
:1012500089CF2685EF1030116DD5EF1010317C400D
:10126000FD177CC07C40E344F0FEFD577CC0224467
:10127000B2409244024941016F10B0481DC17971DA
:101280004ECE52CC06D63E8A22D426D24AD056CA58
:101290005AC85EC6A547BA8963F8E7007370043080
:1012A00001A07370043001A02A8BAE843289B68B02
:1012B000C28A6307082213050006EF2090372A84AC
:1012C000630B05200A09232855034A869305500A13
:1012D0005685EF20505C03C704001C587119230A7F
:1012E000E40203C704003E991379C9FF79C783C795
:1012F0001400A30AF40283C71400E1C383C72400C7
:10130000230BF40283C72400CDCB83C73400A30B87
:10131000F40283C73400D5C383C74400230CF4020E
:1013200083C74400D9CB83C75400A30CF40283C7FE
:101330005400C1C783C76400230DF40283C764004F
:10134000ADCF83C77400A30DF40283C77400B5C783
:1013500083C78400230EF40283C78400B9CF83C7F8
:101360009400A30EF40283C79400A1CB83C7A4000A
:10137000230FF40283C7A400A9C383C7B400A30F3B
:10138000F40283C7B40095CB83C7C4002300F404E0
:1013900083C7C4009DC383C7D400A300F40483C7DC
:1013A000D40081CF83C7E4002301F40483C7E400A1
:1013B00089C783C7F400A301F404930A4400568547
:1013C000A30104042326340323283405232A040418
:1013D000EFF02F9513058401EFF0AF94A947B38781
:1013E0003741232C040400C81CCC40D02322040421
:1013F000232E04045E86DA854A85EFF0AF8D08C09F
:1014000063040A0023208A007370043017F9010076
:10141000130909168327090097F401009384041720
:1014200091C798409C407C4385077CC317F7010017
:101430001307C7141C43850797F6010023A0F61471
:101440009C40C5CB8327090017FB0100130B4B23DE
:1014500089EB9C40DC5763E6F90097F7010023A76E
:10146000871297F701009387A70F9C4317F7010096
:101470001307471048541843850797F6010023A126
:10148000F60E3CC46376A70097F7010023A4A70ECD
:10149000D145EF50A01FD6855A95EFF0EF888327EE
:1014A000090081C79C40FC43B5E38327090005443C
:1014B00099C79C40DC5763F43701EFE03FF5228584
:1014C000B250225492540259F249624AD24A424BD3
:1014D000B24B456182805685EF20D0277D54C5B739
:1014E00013152600EF20F014AA8AE31605DC7D54BC
:1014F000F9B797F7010023AB8708184385476301C5
:10150000F70217FB0100130BAB17A1BF98409440E3
:101510007C43FD177CC3FC42C9FB7360043071B788
:10152000014A17FB0100130BAB15A94B5285D1459E
:10153000EF50C015050A5A95EFE07FFDE3187AFFDA
:1015400097FB0100938B4B205E85EFE05FFC17FA61
:101550000100130AAA205285EFE07FFB17F5010076
:1015600013050521EFE0BFFA17F5010013058521EA
:10157000EFE0FFF917F5010013050522EFE03FF951
:1015800097F7010023A2770197F7010023AC47FFEB
:10159000C9BD411122C406C626C24AC02A8473703E
:1015A000043097F401009384A4FC9C40F9E311E417
:1015B00097F70100938787FD8043130944004A850C
:1015C000EFE01FFB1C5489C713058401EFE05FFAAD
:1015D000CA8517F501001305E51AEFE0FFF497F748
:1015E00001009387E7F9984397F70100938747F73E
:1015F0009C43050797F6010023A4E6F89840850769
:1016000097F6010023AEF6F401CB97F7010093871C
:10161000E7F79843784349EF9C40B1C797F701003B
:101620009387C7F69843630F870873700430984018
:1016300039EB17F70100130727F514439442A5E28D
:101640007D5797F6010023ABE6F0984009CF984309
:10165000784311CB984394437C43FD177CC3FC42F1
:1016600099E373600430B24022449244024941013C
:10167000828097F70100938767F198439C437C43EE
:1016800085077CC32DB794439843F8420507F8C2F9
:1016900017F70100130747EF14439442D5D21843BC
:1016A00058475847584397F6010023A9E6EA71BF07
:1016B000984394437C43FD177CC3FC42B1FF7360A5
:1016C000043099BF97F70100938707E99C4381C7CE
:1016D0007370043001A02244B24092440249410197
:1016E0006FE0DFD241C517F70100130727EA144363
:1016F0008147638BA606411106C622C426C27370B9
:10170000043097F601009386A6E69C4291C71043E9
:101710001C437C4285077CC29C42AA84404981C705
:101720001C43FC43B9E797F701009387E7E59C4327
:10173000638B870497F701009387C7E49C43638416
:10174000870497F70100938727056309F40297F749
:101750000100938727036301F4028547B2402244C6
:1017600092443E85410182803E85828073700430C0
:1017700001A0EF50600545BF9147CDB79C5493B78A
:1017800017008907E1BF8947D1BF7370043097F70D
:1017900001009387E7DD984309EF15C59C43485541
:1017A00081CB97F70100938767DE9843784315E371
:1017B000828017F70100130767DD14431843F842CE
:1017C0000507F8C261FD17F70100130727DC08437E
:1017D000F1B7984394437C43FD177CC3FC42E9FB7B
:1017E000736004308280411122C42A8406C6EFE06F
:1017F000DFCD11E497F70100938747D98043405428
:10180000EFE05FCCB2402285224441018280A547AF
:1018100063F5B7007370043001A0011122CC06CE2D
:1018200026CA4AC84EC652C42A847370043017F9B7
:1018300001001309E9D383270900CDEF71C43C48A7
:101840006388F50817F70100130747D463FCB70056
:101850001443638C860C18434457B3B4950093C467
:10186000140029A00443818C93B41400585463835A
:10187000E70A1C4C2CC863C60700A947B385B740CC
:101880000CCC93172700BA97584897F90100938911
:1018900029DF8A07CE97631AF702130A440052859C
:1018A000EFE01FCD97F701009387C7CC48549C43C6
:1018B00063F6A70097F7010023AEA7CAD145EF4012
:1018C000F05CD2854E95EFE03FC699C0EFE01FB4C3
:1018D0008327090081CB97F70100938727CB9C438F
:1018E000FC439DEBF2406244D2444249B249224A51
:1018F0000561828097F70100938747C998439C430D
:101900007C4385077CC305FC97F70100938707C8D4
:10191000804335B74CD4B1BF6244F240D24442490F
:10192000B249224A05616F40306A814481B725C1BE
:10193000011126CA97F40100938444C59C4006CE49
:1019400022CC4AC84EC6638DA7027370043017F9C3
:1019500001001309E9C18327090091C798409C4001
:101960007C4385077CC3584997F701009387C7E2FA
:101970006302F7028327090081C79C40FC43A5EB63
:10198000F2406244D2444249B24905618280737098
:10199000043001A01C5517F70100130767DDE38B26
:1019A000E7FCE9FB930945002A844E85EFE05FBC24
:1019B00097F70100938707BC48549C4363F6A70040
:1019C00097F7010023A8A7BAD145EF40304C97F70D
:1019D00001009387E7CA3E95CE85EFE0FFB49C40B7
:1019E0005854DC57E368F7F8EFE05FA261B7624450
:1019F000F240D2444249B24905616F40F05C15CDD6
:101A0000011122CC26CA4EC62A8406CE4AC8EFE06F
:101A1000DFAB584897F70100938707D8AA8981441C
:101A20006300F7024E85EFE0FFA9F240624426858D
:101A30004249D244B249056182807370043001A0EA
:101A40001C5417F501001305A5D2E38DA7FCF9FB83
:101A500097F70100938747B09C43A9EB97F70100E4
:101A60009387C7B29C43445413094400DC574A850A
:101A7000B3B4F400EFE0DFAF97F70100938787AFCF
:101A800048549C4393C4140063F6A70097F70100E1
:101A900023A2A7AED145EF40703F97F7010093878F
:101AA00027BECA853E95EFE03FA8ADBF93058401F0
:101AB000EFE09FA785BF0111056506CE22CC26CA9F
:101AC0004AC84EC652C456C25AC0EF208036630E72
:101AD000051AAA8413050006EF20A0352A84630A9C
:101AE000051C05669305500A04D92685EF20A05AE7
:101AF00004588567F117BE94B7474C4593879744C0
:101B0000130A44005CD85285230C0402A301040488
:101B10002326040223280404232A0404EFE07FA0E0
:101B200013058401EFE0FF9FA947232C0404F198DB
:101B300000C81CCC40D023220404232E04040146F8
:101B4000971500009385E5B12685EFE0BF9808C0A2
:101B50007370043017F90100130989A18327090064
:101B600097F40100938484A291C798409C407C43E1
:101B700085077CC317F70100130747A01C4385079F
:101B800097F6010023ACF69E9C40C9C38327090049
:101B900097F901009389C9AE81EB9C40DC5789E736
:101BA00097F7010023A4879E97F701009387479B2F
:101BB000984397F601009386E69B5C549442050790
:101BC00017F60100232EE69838C463F6F60017F7DF
:101BD00001002321F79A139527003E950A05D28527
:101BE0004E95EFE07F948327090081C79C40FC431A
:101BF000DDE78327090091C39C40EF10F04985473A
:101C00006305F50C59E17370043001A097F70100EA
:101C100023AE87961843854797F90100938949A613
:101C2000E314F7F8CE8A17FB0100130BEBB15685CE
:101C3000D10AEFE0DF8DE31C5BFF17F50100130510
:101C4000A5B0EFE0DF8C97FA0100938A2AB15685A0
:101C5000EFE0FF8B17F50100130585B1EFE03F8B37
:101C600017F50100130505B2EFE07F8A17F50100B3
:101C7000130585B2EFE0BF8997F7010023A66791AE
:101C800097F7010023A0579105B7F2406244D24470
:101C90004249B249224A924A024B056182809840E9
:101CA00094407C43FD177CC3FC42A1F77360043071
:101CB00089B76244F2404249B249224A924A024BF1
:101CC0002685D24405616F20E02873700430FD57EB
:101CD00017F701002324F788624497F7010023A92E
:101CE000A788F240D2444249B249224A924A024B62
:101CF00097F7010023A2078805616FE08FDA737000
:101D0000043097F7010023A507866FE0CFE717F7A8
:101D10000100130767841C4385071CC3828073700E
:101D2000043097F701009387A784984305E317F7DA
:101D300001001307678408439C4381CB97F7010098
:101D40009387C7849843784301EF828017F7010097
:101D50001307C78314431843F8420507F8C2C1BFED
:101D6000984394437C43FD177CC3FC42F9FF7360A6
:101D700004308280411106C622C4EFE00FF597E7D8
:101D800001009387677F8043EFE0CFF3B240228565
:101D900022444101828097E701009387277E884390
:101DA0008280797106D622D426D24AD04ECE52CC29
:101DB00056CA5AC85EC697E701009387E7799C43E5
:101DC000B1EF17E701001307277B1C43850797E650
:101DD000010023A3F67A832A0700638F0A0697E798
:101DE00001009387A7779C43814463F1FA0897F930
:101DF00001009389E98817EA0100130A2A798327E9
:101E00000A008546D85793172700BA978A07BE99C4
:101E100083A7090063FFF600854421A897E7010026
:101E20009387C7749C438144850717E70100232FDC
:101E3000F77297E70100938727739C4391C385440A
:101E4000B2502254268502599254F249624AD24A2B
:101E5000424BB24B4561828017E401001304C47207
:101E60001C409C43DDC37370043001A017E40100E3
:101E70001304847197F901009389898017EA01009E
:101E8000130ACA7017EB0100130BCB6E1C409C4366
:101E9000B5C31C40DC4703A9C70083274900930B47
:101EA00049005E8563EEFA04EFE08FEC8327890238
:101EB0001305890199C3EFE0AFEB8327C90203271C
:101EC0000B00DE85139527003E950A054E95637637
:101ED000F70017E70100232FF768EFE0EFE483270F
:101EE0000A000327C902DC57E362F7FA1C40854465
:101EF0009C43C5F3FD5717E701002321F76601B79F
:101F000017E70100232CF764DDBD17E70100130775
:101F100067671C40184397E6010023A7E66617E7AA
:101F200001002321F76697E701009387A7639C438D
:101F3000850717E701002327F7621C409C4399E7B8
:101F4000FD5717E70100232BF76051BD1C40DC470C
:101F5000DC47DC4317E701002322F76049B597E728
:101F600001009387675F984301E77370043001A015
:101F7000011106CE22CC26CA4AC84EC652C456C249
:101F80005AC07370043097E401009384645E9840F3
:101F900061EB98437D1797E6010023AFE65A9C4317
:101FA000D9EB97E701009387675D9C43C9C797EA20
:101FB0000100938AEA6C17EA0100130AAA5B17E989
:101FC00001001309A95C854919A83385EA00EFE0EF
:101FD000AFD5832709005854DC576379F70483A7EA
:101FE0000A0FC1CF83A7CA0FC04713058401EFE0D2
:101FF0002FD8130B44005A85EFE08FD75C5483260B
:102000000A00DA85139527003E950A052A8756951A
:10201000E3FDF6FA17E70100232EF754EFE0CFD0E7
:10202000832709005854DC57E36BF7FA97E7010060
:1020300023AC37536DB701449C4081CB97E7010037
:102040009387C7549C43FC4395E72285F240624442
:10205000D2444249B249224A924A024B05618280E7
:1020600017E701001307875214431843F842050786
:10207000F8C205B7EF404075C9BF17E4010013046B
:10208000E44E1C4095C31C40054999CF193B09C536
:1020900097E7010023AA274D1C40FD1717E7010011
:1020A0002326F74C1C40FDF397E701009387C74BAD
:1020B00098438547E311F7F8EFE04FB50544ADBF0E
:1020C00011CD81E57370043001A017E701001307FB
:1020D000A7481C4399C77370043001A07370043083
:1020E00001A0411122C406C614431841850617E613
:1020F00001002323D64697E601009386E6479442E3
:102100003304B70000C163F7E602637FE40063FDB8
:10211000860097E701009387674788431105EFE042
:102120002FC52285EF4000641D3D01C9B240224405
:1021300041018280E36FE4FCD9BF2244B2404101F7
:102140006FE0CFAC11C917E701001307E7401C434C
:1021500091C77370043001A06FE04FAB411106C608
:1021600022C41843AA87050797E6010023A6E63E86
:1021700097E601009386864117E701001307C73FE2
:10218000184388423304F7001105EFE06FBE228543
:10219000EF40405DE93311E52244B24041016FE078
:1021A000EFA6B240224441018280411122C406C6FA
:1021B00097E701009387473A9C430144850717E757
:1021C0000100232BF73897E701009387273B9C43B7
:1021D00063E0F51217EE0100130E4E5697E2010070
:1021E0009382424901440147854F1303500A21A0BD
:1021F000311E638DC20B83278EFFBA86F5DB8327E2
:10220000CEFFDC43232EFEFE638AC70F03AFC70059
:10221000DC432A97814E232EFEFE6385C70783A8E1
:10222000C70093874803232017015CC383A7880452
:102230002326F7011CC783A7C8021CCB83A7080568
:10224000232C07005CCB03A8080383470800639096
:102250006704C287850783C60700B3850741E38B00
:1022600066FE8981C205C181231EB700850E130752
:10227000070263061F038327CEFFDC43232EFEFEE7
:10228000E39FC7F983274E00232EFEFE49BF8145F9
:10229000231EB700850E13070702E31E1FFD769469
:1022A00013175400311EBA86E397C2F597E7010071
:1022B0009387872D03AE070083270E00639D070ECB
:1022C00097E701009387072C03AE070083270E00D2
:1022D0006392071817EE0100130E8E3A83274E10F3
:1022E0009DE383278E116395072019C223200600E2
:1022F000BD312285B24022444101828083274E00B5
:10230000232EFEFE21B783278E1017EF0100130F37
:10231000EF47DC4317E701002328F7466380E733E4
:1023200083A2C700DC43AA96814E17E70100232D44
:10233000F744914F1303500A6388E70783A8C70047
:102340009387480323A01601DCC283A7880423A631
:10235000F6019CC683A7C8029CCA83A7080523ACC4
:102360000600DCCA03A80803834708006391672AB4
:10237000C287850703C70700B3850741E30B67FEE4
:1023800093D72500C207C183239EF600850E93864E
:1023900006026386122983278E10DC4317E70100AB
:1023A0002324F73EE39CE7F983270E1117E701008A
:1023B000232CF73C61B783274E00130F8E00D443C4
:1023C0002322DE006388E629B307E500D84283A212
:1023D000C600814E2322EE00894F1303500A630684
:1023E000EF068328C7001387480323A01701D8C32B
:1023F00003A7880423A6F70198C703A7C80298CBB0
:1024000003A7080523AC0700D8CB03A8080303479C
:1024100008006318671C4287050783460700B30559
:102420000741E38B66FE13D7250042074183239EB5
:10243000E700850E93870702638D121B83264E00EB
:10244000D8422322EE00E31EEFF80327CE0023221A
:10245000EE0041BF83274E00130F8E00DC43232282
:10246000FE006384E71F83A2C700DC43AA96814E67
:102470002322FE00894F1303500A6306FF0683A838
:10248000C7009387480323A01601DCC283A78804F2
:1024900023A6F6019CC683A7C8029CCA83A7080589
:1024A00023AC0600DCCA03A8080383470800639630
:1024B0006710C287850703C70700B3850741E30B91
:1024C00067FE93D72500C207C183239EF600850EC1
:1024D00093860602638B120F83274E00DC43232270
:1024E000FE00E31EFFF88327CE002322FE0041BF3B
:1024F0008327CE1197EE0100938E8E2ADC4317E7D7
:102500000100232DF7286384D71383AFC700DC4372
:102510003307D500014397E6010023A1F6280D4FAC
:1025200089429308500A6387D707C8479307450332
:1025300008C35CC33C452326E7011CC75C551CCB84
:102540001C5599C3232657003C49232C07005CCB1C
:10255000032805038347080063951705C28785078D
:1025600083C60700B3850741E38B16FF93D7250089
:10257000C207C183231EF700050313070702638AFE
:10258000AF028327CE11DC4397E6010023A8F62093
:10259000E39DD7F983274E1297E6010023A0F6208A
:1025A00069B78147231EF700050313070702E39A63
:1025B000AFFC1A94E31C06D225BB8147239EF6008C
:1025C000850E93860602E39912F117EE0100130EB1
:1025D0002E0B83274E10769493165400E38307D076
:1025E0001DB30147239EE700850E93870702E397FB
:1025F00012E597E701009387E7F803AE07007694AA
:102600009316540083270E00E38607CCA1B58147BB
:10261000239EF600850E93860602E39E12D783273B
:102620008E11769493165400E38107CCD1B583279D
:102630004E1217E701002323F716C1BD83270E11A1
:1026400017E701002322F714E1B98327CE002322E4
:10265000FE0011BD8326CE002322DE00B5B37971C2
:1026600026D24AD04ECE52CC56CA5AC85EC606D6DC
:1026700022D497E90100938929EE17E90100130993
:10268000290017EA0100130AAAEE97EA0100938ACB
:10269000EAEF97EB0100938B6BEE97E401009384D4
:1026A00024EE054B21A883A70900032449108507C0
:1026B00017E701002322F7EA5D3011E89C40E5F7B7
:1026C00083270900E37CFBFEEFD05FD4C5BF7370A6
:1026D000043083270A00B9E383270911C047130593
:1026E0004400EFD0FFE883A70B00FD1717E70100B8
:1026F0002326F7E89C40FD1717E701002322F7E89F
:1027000083270A0089C783A70A00FC4385E308588A
:10271000EF1050042285EF10F0034DB703A70A0015
:1027200083A70A007C4385077CC37DB703A70A0003
:1027300083A60A007C43FD177CC3FC42E9FB73605F
:102740000430F1B797E70100938707E19C43DDE789
:10275000411106C622C426C297E7010023A607E05E
:1027600017E70100130787E21C43B7A6A5A59386C8
:10277000565A9C5B8C43639BD500D0436318B600CC
:1027800094476395C600DC476388D70008430C4331
:1027900093854503EF20E07317E70100130787DDFA
:1027A000144317E401001304A4ED11A81C43A9CF9E
:1027B0001C43FD1797E6010023AEF6DA1443939706
:1027C0002600B6978A07A2979C43EDD30843931738
:1027D0002500AA978A073307F4005443A107A2975C
:1027E000C44244C36385F402DC44B240224417E788
:1027F0000100232DF7D8924441018280854717E7D5
:1028000001002323F7D682807370043001A0C440F6
:10281000D145EF30B067229544C1F9B701114AC8DC
:1028200006CE22CC26CA4EC62A897370043097E49D
:1028300001009384E4D39C4017E40100130404D501
:10284000D9E76314090003290400930949004E8560
:10285000EFD01FD28327890289C713058901EFD0E2
:102860003FD1CE8517E50100130505F3EFD0DFCB8F
:102870009C4081C71C40FC43ADE31C40638B270791
:102880009C409DCF737004309C40C1EB97E70100E2
:10289000938787CF9843184325EBFD5717E701002F
:1028A000232EF7CA9C4089CF1C40FC4391CB184093
:1028B00014407C43FD177CC3FC4299E373600430F1
:1028C000F2406244D2444249B249056182801840D4
:1028D0001C407C4385077CC3ADB7184014407C4343
:1028E000FD177CC3FC42D1FB736004301C40E399AC
:1028F00027F99C40A1C397E701009387E7C59C4354
:10290000ADCB7370043001A09C43DC47DC47DC4353
:1029100017E701002324F7C471B718401C407C431B
:1029200085077CC397E70100938707C69843184340
:102930002DD7D9BF97E70100938747C417E7010058
:10294000130707D49C4303278711631DF700F24048
:10295000624497E7010023AB07C2D2444249B2491F
:10296000056182806244F240D2444249B249056125
:10297000D1BB6244F240D2444249B24905616FD0B2
:10298000FFA83DC9411126C297E40100938404C009
:102990004AC02E898C4006C622C4E105EFD05FBA3A
:1029A00088401105EFD0DFBCFD57630AF90497E7B3
:1029B0000100938767BC804398409C434A9440C37E
:1029C000636CF40497E70100938707BC88438C404D
:1029D0009105EFD0FFB697E70100938727B89C4396
:1029E0006376F40097E7010023AA87B6B240224439
:1029F00092440249410182807370043001A08C40EE
:102A00002244B2409244024917E501001305C5D89B
:102A1000910541016FD05FB197E70100938787B6B9
:102A2000884322448C40B2409244024991054101BE
:102A30006FD01FB111C997E701009387E7B19C439D
:102A400099E77370043001A07370043001A0411144
:102A500026C297E40100938464B39840AE878C400B
:102A6000B7060080D58F06C622C41CCFE10532848C
:102A7000EFD09FAB88401105EFD09FAFFD57630E9D
:102A8000F40097E70100938727AF8843B240924450
:102A90002295224441016F30F04C8C402244B240D8
:102AA000924417E50100130525CF910541016FD030
:102AB000BFA725CD411126C297E40100938404AD40
:102AC0004AC02E898C4006C622C4E1053284EFD06C
:102AD000BFA588401105EFD0BFA98547630AF4045C
:102AE00097E70100938747A9804398409C434A9405
:102AF00040C3636CF40497E701009387E7A8884319
:102B00008C409105EFD0DFA397E70100938707A5DD
:102B10009C436376F40097E7010023A187A4B240A9
:102B2000224492440249410182807370043001A022
:102B30008C402244B2409244024917E5010013053B
:102B4000A5C5910541016FD03F9E97E7010093878E
:102B500067A3884322448C40B240924402499105C5
:102B600041016FD0FF9D411106C622C426C25C45BB
:102B7000C04735CC930484012685EFD07F9F97E72B
:102B800001009387679D9C43B5E793044400268525
:102B9000EFD01F9E97E701009387C79D58549C4331
:102BA00063F6E70097E7010023A6E79C9317270049
:102BB000BA978A0717E50100130585ACA6853E95EF
:102BC000EFD09F9697E701009387479C9C4358540A
:102BD0000145DC5763F8E700854717E70100232527
:102BE000F7980545B24022449244410182807370B7
:102BF000043001A0A68517E50100130565B7EFD0E5
:102C0000BF92C9B797E70100938707959C4381E777
:102C10007370043001A0411106C622C426C2B70752
:102C200000804045CD8F1CC12DC4EFD07F9493040C
:102C300044002685EFD0DF9397E7010093878793C1
:102C400058549C4363F6E70097E7010023A4E792FA
:102C500093172700BA978A0717E50100130545A2C5
:102C60003E95A685EFD05F8C97E70100938707928A
:102C70009C4358540145DC5763F8E700854717E744
:102C800001002323F78E0545B240224492444101BE
:102C900082807370043001A011CD97E70100938703
:102CA000678C984397E701009387078D9C4318C171
:102CB0005CC182807370043001A055C1D1CD411137
:102CC00006C622C42A877370043097E801009388EF
:102CD000288A83A7080091CB97E701009387078B89
:102CE00094439C43FC428507FCC217E30100130395
:102CF000A3889C4103260300FD560144638FD7023D
:102D000017EE0100130E0E8603250E0003280700A0
:102D100054436305A80005446371D6023308D640C6
:102D20000544637CF80003250E00918F0326030001
:102D3000B6979CC108C350C3014483A7080081CB48
:102D400097E70100938787849C43FC4381EF2285AA
:102D5000B2402244410182807370043001A073703C
:102D6000043001A0EF305026DDB7854717D70100AA
:102D7000232CF77E828019C16845828001458280BC
:102D800011C16CC5828097E7010093872780884333
:102D9000828097D701009387A77D9C43054589CB07
:102DA00097D701009387477B8843133515000605A5
:102DB000828031CD011126CA97D401009384047D0D
:102DC0009C4006CE22CC4AC84EC65855DC57637983
:102DD000F7021C4D63C707009C40D457A947958F45
:102DE0001CCD93172700BA97584917E9010013091A
:102DF00029898A07CA97630DF7009C40DC575CD588
:102E0000F2406244D2444249B249056182808280E4
:102E1000930945002A844E85EFD08FF59C4017D743
:102E20000100130727751843DC575CD46376F7005D
:102E300017D701002320F774139527003E956244AD
:102E40000A05F240D244CE854A95B249424905610D
:102E50006FD08FED19CD411106C622C426C297D777
:102E600001009387A77280436307A4007370043046
:102E700001A0014582807C4881E77370043001A085
:102E800054543848FD177CC86383E60099C7014550
:102E9000B24022449244410182809304440026853A
:102EA000EFD00FED284897D701009387A76C984380
:102EB000A947898F48D41CCC6376A70097D7010017
:102EC00023AAA76AD145EF30607C97D7010093878A
:102ED000277B3E95A685EFD02FE5054555BF73703E
:102EE000043097D701009387A7689C4391CB97D76D
:102EF00001009387A76998439C437C4385077CC363
:102F0000828097D701009387A7669C438DC397D78C
:102F100001009387A7679843784311CB9843944364
:102F20007C43FD177CC3FC4299E3736004308280CC
:102F300097D7010093878765904394439843A947A7
:102F4000D456084E958F1CCF828097D70100938767
:102F5000E763984309C79443F84A0507F8CA8843CA
:102F6000828079714AD006D622D426D24ECE2A89C2
:102F70007370043097D401009384845F9C4017D40D
:102F800001001304A460BDE31C40BC4F89E71C4052
:102F90000547F8CFD1E19C4081C71C40FC43F1EBD1
:102FA000737004309C408DEF1C40A84F11C5630422
:102FB00009021C4023AC07041C4023AE07049C40BC
:102FC00081C71C40FC438DEBB250225492540259ED
:102FD000F2494561828018403C4FFD173CCFE9BF64
:102FE00018401C407C4385077CC37DBF18401C40B3
:102FF0007C4385077CC349BF184014407C43FD17C0
:103000007CC3FC42F1F373600430B25022549254FA
:103010000259F2494561828008402EC61105EFD061
:103020002FD5B245FD576380F50697D701009387EA
:10303000A75483A9070018409C43AE992322370167
:1030400063ECF90497D701009387075488430C4039
:103050009105EFD0EFCE97D70100938727509C437F
:1030600063F6F90097D7010023AA374FEFD00FBAC4
:103070001DB7184014407C43FD177CC3FC428DF300
:103080007360043031BF0C4017D501001305C570C3
:103090009105EFD06FC9D9BF97D701009387874EAD
:1030A00088430C409105EFD0AFC9C9B779714AD0B8
:1030B0004ECE06D622D426D252CC2E89B289737037
:1030C000043097D401009384A44A9C4017D4010093
:1030D0001304C44BF9EF18408947784F630CF7008D
:1030E0001C401345F5FFB84F798DA8CF1C4005470C
:1030F000F8CFADE69C4081C71C40FC43F5E37370FC
:1031000004309C40B1E7638609001C40BC4F23A0FB
:10311000F900184085470145784F630BF7001C40C4
:103120001349F9FF0545B84F3379E90023AC27056A
:103130001C4023AE07049C4081C71C40FC43C1E3F4
:10314000B250225492540259F249624A4561828037
:1031500018401C407C4385077CC375B7084036C6C1
:103160001105EFD0EFC0B246FD576385F60897D73B
:1031700001009387674003AA070018409C43369AD2
:10318000232247016363FA0897D701009387C73F5B
:1031900088430C409105EFD0AFBA97D701009387D1
:1031A000E73B9C436370FA0697D7010023A8473B8F
:1031B00091A818401C407C4385077CC329BF184058
:1031C00014407C43FD177CC3FC42BDFB736004309C
:1031D000B250225492540259F249624A45618280A7
:1031E000184014407C43FD177CC3FC4289FB73608C
:1031F000043031B70C4017D501001305E55991058E
:10320000EFD08FB2EFD08FA0F5B597D7010093879D
:10321000673788430C409105EFD08FB2E5B751C1B5
:10322000411106C622C426C24AC07370043097D426
:1032300001009384E4339C40B9EB99C23C4D9CC29D
:10324000B2878946704D74CD2E872A846386D7064F
:1032500063FCF6048D456387B70091456395B7001D
:103260006300D60C38CC8547630FF60405449C40B8
:1032700081CB97D70100938767319C43FC43A9E337
:103280002285B2402244924402494101828097D76C
:1032900001009387A72F98439C437C4385077CC3F9
:1032A00069BF7370043001A08546E39ED7FA3C4D98
:1032B00033E7B70038CD45BF3C4D85073CCD65B7FA
:1032C000EF30805075BF130944004A85EFD04FAAF4
:1032D00097D701009387072A48549C4363F6A700B9
:1032E00097D7010023A8A728D145EF30203A97D7D8
:1032F00001009387E7383E95CA85EFD0EFA21C54B2
:1033000081C77370043001A097D701009387072805
:103310009C435854DC57E3FBE7F4EFD02F8FB9B749
:103320000144B1B739CD011122CC26CA4AC84EC6D4
:1033300052C456C206CEBA89368AB2842E892A84ED
:10334000EFD0AF98AA8A63050A003C4C2320FA000C
:10335000784C89477CCC6389F40263F4970C8D46E2
:103360006387D40091466396D400630AF70A232C3E
:1033700024058547631EF7061C5499CB73700430EF
:1033800001A07370043001A03C4C85073CCCD5B73C
:1033900097D701009387471C9C43ADEB93044400EF
:1033A0002685EFD0EF9C97D701009387A71C485440
:1033B0009C4363F6A70097D7010023ADA71AD14518
:1033C000EF30C02C97D701009387872BA6853E95B9
:1033D000EFD08F9597D701009387471B9C43585494
:1033E000DC5763F7E70063850900854723A0F900F0
:1033F00005445685EFD00F8D2285F2406244D244B9
:103400004249B249224A924A056182809305840169
:1034100017D501001305C535EFD00F9165BF0144E5
:10342000C9BF8547E397F4F43C4C33E92701232CCB
:10343000240581B74DC1011122CC26CA2A844EC66B
:1034400006CE4AC8AE84EFD04F888947744C7CCCF6
:103450003C4C0547AA8985073CCC6395E6061C547D
:1034600081C77370043001A097D701009387C70EFE
:103470009C43ADE7130944004A85EFD06F8F97D77F
:1034800001009387270F48549C4363F6A70097D702
:10349000010023A1A70ED145EF30401F97D70100AF
:1034A0009387071ECA853E95EFD00F8897D70100F6
:1034B0009387C70D9C435854DC5763F5E70099C0C8
:1034C00085479CC06244F240D24442494E85B2498D
:1034D00005616FC03FFF7370043001A09305840144
:1034E00017D501001305C528EFD00F84C1B7AA87EF
:1034F00029C57370043017D70100130767071443F9
:103500009DE2F04F894601456315D60023AE0704BE
:1035100005451C4381CB97D7010093872707984324
:10352000784315E3828097D6010093862606904261
:1035300094427442850674C2E9B797D70100938715
:10354000E7049C437DB7984394437C43FD177CC3B9
:10355000FC42E9FB7360043082805D71A6C2CAC080
:1035600052DC56DA5AD85ED686C6A2C44EDE62D483
:1035700066D26AD017D901001309490217DB01008E
:10358000130B0B0197D401009384C40097DA010058
:10359000938A8A00054AA54B832709009843630153
:1035A0000712DC4783A90700EFE06FF6EFE02FF783
:1035B00083270B002A8C6362F50A97D7010023A9A1
:1035C000A7FC01466370351B8840B3858941EFD065
:1035D000DFBDEFE0DF9863010512884081460146B8
:1035E0002C00EFD0EFEB4DD9A247E3C807FEC2494C
:1035F00083A7490189C713854900EFC07FF7EFE032
:103600000FF283270B002A8C636DF508A24717D7AA
:103610000100232F87F7E3E2FBFCB317FA0013F74F
:103620000721631A071613F7770C6318071E93F721
:103630000702C5D74E85EF00F01145B7DC47C047FC
:1036400083AC0700930944004E85EFC07FF25C50C5
:10365000228582975C4C6384470B8327090098433B
:1036600071FF03A70A0097D6010023A386F397D61C
:10367000010023A3F6F297D7010023A1E7F2EFE0C0
:103680001F8EA1BFDC47C04703AD0700930C440069
:103690006685EFC0FFED5C50228582975C4C6386A7
:1036A000470983270900984371FF03A70A0097D6AB
:1036B000010023A3F6EE97D7010023A1E7EEB9B7E7
:1036C000EFE0EFE4EFE0AFE583270B002A8CE36641
:1036D000F5F883A70A00884081499043B385894162
:1036E00017D70100232687EB13361600EFD0FFAB68
:1036F000EFE0FF86E31305EEEFC05FD1F9BD1C4C90
:10370000CE85E69763E9FC049C4089CF02CA66CC6B
:1037100022CEEFF00FE88840814601464C08EFD0FA
:103720000F8805FD7370043001A01C4CE685EA97F4
:10373000636CFD049C4089CF02CA6ACC22CEEFF0B4
:103740004FE58840814601464C08EFD04F8531F95E
:103750007370043001A0032509005CC000C8EFC0ED
:103760003FDEE5BDEFE0AFFF83270900DC47C04740
:10377000930C44006685EFC0BFDF5C4C638F47034A
:103780005C502285829791BD032509005CC000C86A
:10379000EFC01FDB39B7B24723ACF900A5CFE297E2
:1037A00023A2F90023A8390193854900636FFC0423
:1037B00003A50A00EFC0DFD80DB51C4C00C8338745
:1037C000F90058C0636DEC02330C3C416363FC02AA
:1037D0009C4089CF02CA4ECC22CEEFF08FDB8840CE
:1037E000814601464C08EFC09FFB59F973700430C5
:1037F00001A003A50A00E685EFC09FD451B70325B9
:103800000900E685EFC0DFD3A5BF03250900EFC09F
:103810003FD3E1B37370043001A0B24783A689019E
:1038200023A839013387D70023A2E9006364EC049D
:10383000B307FC4063EBD70483A749024E85829708
:1038400083A7C901E39B47D983A68901B247984062
:10385000B69711CF02CA3ECC4ECEEFF08FD3884040
:10386000814601464C08EFC09FF3E31805D67370FC
:10387000043001A06374FC00E370F7FC0325090029
:1038800093854900EFC0DFCB89BB03A50A00938570
:103890004900EFC0FFCA91B3411122C406C626C237
:1038A0004AC017D401001304E4CEEFF04FE31C40EC
:1038B00095CBEFF00FE51C409DC38148014881473F
:1038C000094781461306004097D50100938505AF4F
:1038D000170500001305A5C8EFD05F9A39E973708A
:1038E000043001A017D90100130949EC4A85EFC043
:1038F0001FC297D401009384A4EC2685EFC03FC17A
:103900000146B145114597D7010023A927C997D78B
:10391000010023A397C8EFC07FDB17D70100232B3B
:10392000A7C611CD97D501009385C5A8EFD0AFFCF0
:1039300049B7B240224492440249410182807370E7
:10394000043001A0A5C9797156CAAA8A1305C0021C
:1039500022D426D24AD04ECE52CC06D65AC85EC603
:103960003A89B689328AAE84E9212A8405C9EFF002
:103970000FD797D701009387E7C19C439DCFEFF006
:103980004FD8130544002320540104CC232E4401B6
:103990002320340323222403EFC0BFB82285B25072
:1039A000225492540259F249624AD24A424BB24BD3
:1039B000456182807370043001A097DB0100938B16
:1039C000EBDE5E85EFC0BFB417DB0100130B4BDFEE
:1039D0005A85EFC0DFB30146B145114597D70100C5
:1039E00023AE77BB97D7010023A867BBEFC01FCEDC
:1039F00017D701002320A7BA01C997D501009385E5
:103A0000659BEFD04FEFA5BF7370043001A039C59F
:103A1000011122CC06CE26CA17D40100130484B7A4
:103A2000832804002A88014563850802BA842EC2CF
:103A3000368732C442C6954663C5B602EFF06FB50D
:103A40008947630BF5020840814601464C00EFC0F0
:103A50001FD5F2406244D244056182807370043005
:103A600001A04C0081463A864685EFD08F88F2400F
:103A70006244D244056182800840814626864C001B
:103A8000EFC0FFD1F9B719C10841828073700430CB
:103A900001A001E57370043001A0411106C622C4E3
:103AA0002A84EFF0CFC348483334A000EFF06FC54D
:103AB0002285B24022444101828001E573700430C6
:103AC00001A0411122C42A8406C6EFF04FC1005064
:103AD000EFF02FC3B240228522444101828001E5EC
:103AE0007370043001A0411122C426C22E84AA841E
:103AF00006C6EFF0CFBE80D02244B24092444101CE
:103B00006FF02FC04111714522C406C61D262A84BC
:103B100011C5232005001105EFC07F9F2285B2400B
:103B200022444101828001CDB70700FFED8F81C79C
:103B30007370043001A099E57370043001A07370B4
:103B4000043001A0011122CC4AC84EC652C456C24C
:103B500006CE26CABA893689B28A2E842A8AEFF01E
:103B60004FA311E5638509007370043001A0EFE0F5
:103B70000F9A83240A00B37794006316090295C74D
:103B800063870A009347F4FFE58F2320FA00EFE0F4
:103B90000FBDF240624426854249D244B249224ACE
:103BA000924A05618280E30DF4FCE38209FEB3359D
:103BB0005001E20563050900B7070004DD8D4E865C
:103BC000C18D13054A00EFE0FFE6EFE04FB919E1C0
:103BD000EFC0DF83EFF0CFB593176500AA8963D8F4
:103BE0000700B7040001FD14B3F499005DB7EFF0CE
:103BF0000FAF83290A00B3773401631E090089CB14
:103C000063880A009347F4FFB3F737012320FA00D3
:103C1000EFF02FAFF9B7E31DF4FEDDB701C9B70729
:103C200000FFED8F99C77370043001A073700430EA
:103C300001A0411122C42A8406C626C24AC02E8988
:103C4000EFF0EFA904409345F9FFB3F795001CC0CE
:103C5000EFF02FABB2402244268502499244410145
:103C60008280411122C42A8406C6EFC01F8600400C
:103C7000EFC05F85B240228522444101828009C99C
:103C8000370700FFB3F7E50099C77370043001A050
:103C90007370043001A06F20F034B70700FFF18F7C
:103CA00081C77370043001A001E67370043001A075
:103CB000011122CC4AC84EC652C406CE26CA368945
:103CC000AE892A8A3284EFF0CF8C21E163050900A6
:103CD0007370043001A0EFE08F8383240A00CE8547
:103CE0005285B3E49900613FB37794006307F4060B
:103CF00083240A00EFE0AFA6F240624426854249E1
:103D0000D244B249224A05618280EFE04F80832489
:103D10000A00CE855285B3E434019537B3F78400A9
:103D2000638D8702E30609FCB70500054A86C18D4D
:103D300013054A00EFE01FD0EFE06FA219E1EFC0DA
:103D4000EFECEFF0EF9E93176500AA8463DF0700A6
:103D5000B7070001FD17FD8C45B783270A00134400
:103D6000F4FFE18F2320FA0071B7EFF04F9783241F
:103D70000A00B3779400639787009347F4FFE58FB9
:103D80002320FA00EFF0EF97E1B7411122C406C6F5
:103D90002A8426C2EFD0BFF75C4085C3084893044D
:103DA000C4006316950015A0084863009502B70586
:103DB0000002EFE03FE55C40E5FB2285612A2244FA
:103DC000B240924441016FE08F997370043001A0BA
:103DD00009C9370700FFB3F7E50099C773700430CE
:103DE00001A07370043001A06F20D01F01C9B70774
:103DF00000FFED8F99C77370043001A07370043019
:103E000001A0411122C426C206C62A84AE84EFF066
:103E10000F8D184093C7F4FFF98F1CC02244B240A5
:103E2000924441016FF0EF8D19C1084D8280014528
:103E30008280411122C406C62A84EFD05FED97C765
:103E400001009387E7759C43A1EBE56717D7010055
:103E500013078798F11797C6010023A9E67417C7BF
:103E600001002323F77417D701002329F79697C77A
:103E700001009387277317D70100232FF7948547F5
:103E800017C701002326077217C70100232C0770EC
:103E900017C701002326F77019E8EFE04F8CEF10E9
:103EA000C00201442285B2402244410182801305B0
:103EB000840093773500C1EFE5671307F5FFE91735
:103EC000E3EDE7FC97C601009386466E9C4229A06D
:103ED000984311C7BE86BA87D843E36BA7FE17C7BE
:103EE00001001307276CE38AE7FA984341461384DD
:103EF000870098C2D843B306A7406378D6023388B8
:103F0000A7002322D800C8C38325480097C6010014
:103F10009386C66911A0BA8698425043E36DB6FEF7
:103F20002320E80023A00601D84397C70100938708
:103F3000276B9C43998F17C701002323F76AEFE093
:103F40000F8231DC2285B240224441018280719986
:103F500011059DB729C9411122C406C62A84EFD094
:103F60001FDB930584FF0326C4FF17C70100130757
:103F7000E76311A03E871C43D443E3EDC6FE232C28
:103F8000F4FE0CC397C70100938787659843832786
:103F9000C4FF2244B240BA9717C701002322F76436
:103FA00041016FD0DFFB828097C701009387476391
:103FB0008843828082803367B5000D8BAA871DE716
:103FC0009308D6FFAA982A87AE866371150303A8C3
:103FD000060011079106232E07FFE36A17FF934798
:103FE000F5FFC697F19B9107BE95AA972A9663F3B2
:103FF000C70A9386450013884700B3B6D70033B885
:10400000050133E7F50093C61600134818000D8B21
:10401000B3E6060113371700758F330EF64093860B
:10402000170029CF1337AE0031EB13532E002E8823
:10403000BE860147832808000507110823A0160142
:104040009106E36967FE1377CEFFBA95BA976302CC
:10405000EE0483C60500138717002380D700637A18
:10406000C70283C6150013872700A380D700637299
:10407000C70203C725002381E7008280B307F6400B
:10408000AE97850503C7F5FF8506238FE6FEE39A05
:10409000F5FE82808280B367C5008D8BB308C500B2
:1040A000E9C36371150FB307A0408D8B13873700E9
:1040B000954693F5F50F130815003383A8407D1638
:1040C0006373D70015476363E60CD5CF2300B500B3
:1040D0000547638DE700A300B5000D4713082500D1
:1040E0006396E700130835002301B5001396850099
:1040F0004D8E13970501518F3303F340939685013D
:10410000D98E13562300AA97014794C30507910738
:10411000E36DC7FE1377C3FFB307E8006307E30649
:104120002380B70013871700637C1703A380B700B1
:1041300013872700637617032381B700138737009F
:1041400063701703A381B70013874700637A1701D1
:104150002382B7001387570063741701A382B70047
:10416000828093F5F50F13978500D98D139705017C
:104170004D8FE37715FFAA87910723AEE7FEE3EDA6
:1041800017FF828082802A8895B78280AA8749BFDC
:10419000834705002A8799C7050583470500EDFF7A
:1041A000198D82800145828005058347F5FF8505CD
:1041B00003C7F5FF91C7E389E7FE3385E7408280B7
:1041C0008147E5BFAA87850503C7F5FF8507A38F4C
:1041D000E7FE75FB82808346050093070002639724
:1041E000F600050583460500E38DF6FE938756FD30
:1041F00093F7D70F85C7AA87814585CE01458507E7
:10420000138606FD1317250083C607003A95060599
:104210003295F5F699C13305A0408280938536FD2D
:104220008346150093B5150093071500E1FA014583
:10423000D5B7014582809C412380A7009C4185071A
:104240009CC1828097C601009386C6369C42175750
:1042500003001307275B13861700BA972380A70074
:1042600097C5010023A8C534A9476308F500930743
:1042700000046305F6000145828075DE370610F004
:1042800005078347F7FF2320F6F09C42FD1797C5EB
:10429000010023A1F532EDF7014582804D71232203
:1042A000911423202115232A51132324811323261B
:1042B000111423248114232E3113232C411323287A
:1042C000611323267113232291132320A113232E7C
:1042D000B111AA842E8932C6130C5002A54A834715
:1042E000090063808703B9CB804011A0A1CB2300D4
:1042F000F40080400509050480C083470900E39766
:1043000087FF0346190093081900C686130D0002A3
:10431000FD597D5A0148130550059307D6FD93F7C3
:10432000F70F138916006363F52A17C701001307F7
:1043300067CD8A07BA979C43BA9782878320C114B6
:104340000324811483244114032901148329C113F4
:10435000032A8113832A4113032B0113832BC112D8
:10436000032C8112832C4112032D0112832DC111C4
:1043700071618280A14C02C4854763D50715B2479D
:104380008040938B770093F68BFF03AB060083A9E5
:104390004600938786003EC6668681465A85CE854E
:1043A000EF10D05E2AC8814763853723930D410102
:1043B000854B668681465A85CE85EF10607F8146A3
:1043C00066862A8BAE89EF10705CA24723A0AD00F1
:1043D00093861B00910D63843701B68BD9BFE37EB2
:1043E0009BFF63DD4601A2872380A70180407D1AE1
:1043F000930714009CC03E84E3C846FF93962B00AD
:104400001C08BE9631A8938777052300F4008040EE
:10441000FD1B93871B00050480C0F116E351F0ECEF
:104420009C42E3E2FAFE93870703C5B79C409306DC
:10443000000332472380D7009C4093064700C14CBD
:104440001386170090C013068007A380C700804022
:1044500002C4BA87050480C003AB0700814936C691
:1044600025BFB24783AC0700938B470063840C1CC5
:10447000635F40199307D0026319FD1683C70C00D0
:1044800085C363DC09189440850C7D1A2380F600EF
:104490008040050480C083C70C00E5F7635D4001E0
:1044A0008040930700022300F40080407D1A050439
:1044B00080C0E31A0AFE5EC61DB502C48547A94C3A
:1044C000E3CF07EBB24780409386470071B703C63E
:1044D0001600CA8699B59C40930650022380D700E7
:1044E0008040050480C0E5BBC14C02C471B5B24731
:1044F00003C61600CA8683A9070091073EC6E35E7D
:104500000AE04E8AFD5911BD03C61600130DD002F4
:10451000CA8621B59347FAFFFD8703C61600337A92
:10452000FA00CA86DDBB03C61600130D0003CA8657
:10453000EDB383C51600930906FDCA86938705FD72
:104540002E86E3EEFAFA93972900BE99850686092E
:10455000AE9983C50600938909FD938705FD2E86D4
:10456000E3F3FAFE69BF32479C40144311073AC691
:104570002380D7008040050480C095B3854763D36E
:10458000070BB24793867700E19A938786003EC671
:1045900083A946009C4263DC090A94401306D002BA
:1045A000B307F0402380C6008040B336F000B30963
:1045B0003041050480C03E8BB389D940A94C02C468
:1045C000E1BB03C616000508CA8681BB9C4046892C
:1045D00021B7E37D9BDD8547814B8546E3C547E1F8
:1045E00031BD97CC0100938CECDDCE856685EF1054
:1045F0006004330AAA40635C400180402300A401A8
:1046000080407D1A050480C0E31A0AFE014A83C770
:104610000C00E38207EAE3C809E6FD197D57E3943D
:10462000E9E6ADBDB247938647009C4336C693D9B1
:10463000F74195B7635640019307D002E313FDFAA3
:1046400097CC0100938C0CD8930780021DBD3E8B44
:10465000A94C02C4804089B34D71232E3113B70990
:1046600000409387F9FF2324811423229114232CE3
:104670004113232A51132326111423202115232803
:1046800061132326711323248113232291132320E2
:10469000A113232EB1112A8A2EC417C401001304BA
:1046A00064F1975A0300938AEA1597C40100938432
:1046B000E4AA3EC693055002294513080004B70634
:1046C00010F083470A006386B704C1C71840050A83
:1046D00013061700569797C8010023ADC8EC2300B6
:1046E000F7006382A706E31E06FD175703001307B2
:1046F000671105078347F7FF23A0F6F01C40FD175D
:1047000017C601002328F6EAEDF783470A00E39E67
:10471000B7FA83461A0013051A002A87930B000282
:104720007D5B7D5C014893055005A5489387D6FDC8
:1047300093F7F70F130A170063E7F5348A07A69774
:104740009C43A6978287175703001307A70B55F2C0
:104750008DBF8320C11403248114832441140329B1
:1047600001148329C113032A8113832A4113032BC4
:104770000113832BC112032C8112832C4112032DB0
:104780000112832DC11171618280A14C014D8547B9
:1047900063DB0719A2479D07E19B83AD070003ABCD
:1047A0004700138787003AC4668681466E85DA859E
:1047B000EF10D01D2AC863066D35130941018549E4
:1047C000668681466E85DA85EF10803E6686814674
:1047D000AA8D2E8BEF10901B2320A90085091109AB
:1047E000E3106DFFE3FE9DFD13060004B70610F015
:1047F00063D189031C4013871700D69797C5010022
:1048000023AAE5DA23807701630CC7047D1CE3C388
:1048100089FFB2476800A548B386F9008A061C08DC
:10482000BE96294813030004370610F0E384A6E877
:104830009C429305000363F4F8009305700518404B
:10484000AE9793051700569717CE01002324BED6C6
:104850002300F7006380072B638C6526F116F9B7F8
:1048600017570300130707FA05078347F7FF23A02D
:10487000F6F01C40FD1797C5010023ADF5D2EDF70A
:104880007D1C71B71C40130600041387170097C5E1
:10489000010023A1E5D2B386FA009305000323802B
:1048A000B6006300C73E890797C6010023A4F6D06F
:1048B0005697930680072300D70017570300130766
:1048C00067F4B70610F0639EC70005078347F7FF3C
:1048D00023A0F6F01C40FD1717C60100232CF6CCD0
:1048E000EDF7A247C14C014D91072247014B832DA3
:1048F00007003EC455BDA24783AC0700138947009B
:10490000638F0C3A635480219307D002639EFB2E81
:1049100003C70C00BA856310072025AC8547A94C56
:10492000014DE3C907E7A2479107C1B7A2478346F4
:104930001700528703AB070091073EC4E3580CDE13
:104940005A8C7D5BE5B383461700930BD0025287E8
:10495000F1BB9347FCFFFD8783461700337CFC00C7
:104960005287E9B383461700930B000352877DBB40
:1049700003461700138B06FD5287930706FDB28688
:10498000E3EEF8FA93172B00DA9705078607B2973C
:1049900003460700138B07FD930706FDB286E3F37A
:1049A000F8FE69BFA2451C4029469841938617002E
:1049B000D69717C50100232FD5BE2380E7001389A2
:1049C00045006301C72A930700046387F6204AC4A1
:1049D000D5B1854763DF0729A24713877700619B1D
:1049E000930787003EC4032B47001C43635B0B30D7
:1049F0001840130600049306170097C5010023AB67
:104A0000D5BA56979305D0022300B7006388C62C09
:104A1000B307F0403337F000330B6041BE8D330BEA
:104A2000EB40A94C014D49B3834617000508528756
:104A3000F5B9834617005287D5B91C409306000488
:104A40001387170017C601002326E6B6D69713066C
:104A500050022380C700E31FD7C417570300130772
:104A600067DAB70610F005078347F7FF23A0F6F0D3
:104A70001C40FD1717C60100232EF6B2EDF71DB935
:104A8000C14C014D29B31C40930600042A8A1387A8
:104A9000170017C60100232FE6B0D6971306500261
:104AA0002380C700E318D7C017570300130787D523
:104AB000B70610F005078347F7FF23A0F6F01C4068
:104AC000FD1717C601002327F6AEEDF72A8ADDB6DB
:104AD00017570300130707D305078347F7FF232062
:104AE000F6F01C40FD1797C5010023A5F5ACEDF7C6
:104AF000F1162DBB175703001307C7D0F1FDF116B0
:104B000035B3E3FC9DCB8549C5B1014C03C70C000F
:104B1000BA85E30E07EAFD58294513080004B706D5
:104B200010F063570B0A1C4013861700D69717C363
:104B300001002321C3A82380E7006384A506630442
:104B40000609850C03C70C007D1CBA8579FBE35070
:104B500080E91C409305000213060004B70610F01C
:104B600021A07D1CE3050CE613871700D697238050
:104B7000B70017C50100232FE5A2BA87E313C7FECC
:104B800017570300130707C805078347F7FF23A03C
:104B9000F6F01C40FD1717C50100232DF5A0EDF719
:104BA000C9B7175703001307E7C541DE0507834759
:104BB000F7FF23A0F6F01C40FD1717C60100232BBA
:104BC000F69EEDF7BDBF175703001307A7C3F9BF44
:104BD0007D1BE31A1BF5A5BF17570300130787C2F8
:104BE000B70610F005078347F7FF23A0F6F01C4037
:104BF000FD1717C60100232FF69AEDF74AC45DBCD6
:104C000097BC0100938C0C7CDA856685EF009022BE
:104C1000330CAC40E35C80EF1C4013060004B70685
:104C200010F021A07D1CE3020CEE13871700D6972D
:104C30002380770197C5010023AEE596BA87E31379
:104C4000C7FE175703001307E7BB05078347F7FFA6
:104C500023A0F6F01C40FD1797C5010023ACF59486
:104C6000EDF7C9B7175703001307C7B9B5FA4AC418
:104C700091B4A247138747009C433AC413DBF74122
:104C8000B5B3175703001307E7B7B70610F00507CA
:104C90008347F7FF23A0F6F01C40FD1717C601005D
:104CA000232AF690EDF7854717C701002324F790D4
:104CB00093078007175703002306F7B41DB1635607
:104CC00080019307D002E39DFBF297BC0100938C17
:104CD0006C6F130780029305800235BD9756030061
:104CE000938646B2370610F0850603C7F6FF2320E9
:104CF000E6F018407D1797C5010023ADE58A6DF7F2
:104D000001BBBE8DA94C014D45B4B70710F023A0DF
:104D1000A7F201A03971130341022ED29A8506CE63
:104D200032D436D63AD83EDA42DC46DE1AC62D32C6
:104D3000F2400145216182805D711303810322D419
:104D40002AC632DC2A841A86680006D6BEC236DE3F
:104D5000BAC0C2C4C6C61ACEEFF04FD4B247238041
:104D600007003245B250018D225461618280B7073D
:104D700010F083A647F403A607F403A747F4E31A49
:104D8000D7FE8966938606F4B29633B6C600B3059D
:104D9000E60023A4D7F423A6B7F48280B70710F067
:104DA00003A747F403A607F483A647F4E31AD7FE44
:104DB0008966938606F4B29633B6C60023A4D7F468
:104DC000B305E60023A6B7F49307000873A04730A5
:104DD0008280411122C406C697B701009387077EDF
:104DE00017B401001304447D98431C401306F07C63
:104DF000930647069387470697B5010023A0D57C05
:104E000097B5010023AAF57A6346D600B240224442
:104E1000410182801307478997B7010023A0E77AF1
:104E2000EF00C07A8547631FF500184085679387B8
:104E3000F7760145E3DCE7FCC93D2244B24041017D
:104E40006FC0FFEB17B5010013054558E135094563
:104E50006D3D2244B24041016FC07FEA17B50100A9
:104E6000130585586FF01FEB17B501001305455862
:104E70006FF05FEA411122C426C206C6856417B4EA
:104E8000010013046457938784380100FD17F5FF70
:104E90002285EFF03FE8C5BF014585A5411106C653
:104EA000EF00C072054781476316E500B2403E85BA
:104EB0004101828017B5010013054551EFF09FE5D0
:104EC000B24089473E85410182807370043001A061
:104ED00082807370043001A0411122C406C617B449
:104EE00001001304E46E0145EFD05F931C40850779
:104EF00017B70100232EF76CFDB7411122C426C25B
:104F000006C6AA8405440145EFD05F9181467D56CF
:104F100081452685EFB0DFD8814601468145630093
:104F20008502268597B7010023AA876AEFB03F87DD
:104F3000E30B85FC97B7010023A2876AE9B7814696
:104F4000014681452685EFB09F85E30E85FA97B728
:104F5000010023A5876845BF797156CAAA8A05450D
:104F600006D622D426D24AD04ECE52CC5AC85EC6DD
:104F700062C4EFB0FFAD35C9AA8917BA0100130AA0
:104F8000EA6417BC0100130C2C6497B401009384ED
:104F9000246497BB0100938BEB630544094B0D49D7
:104FA0008146014681455685EFB09FCF6306850057
:104FB00097B7010023A48762014597B7010023A991
:104FC0000760EFC08FFC09C597B7010023A8876071
:104FD00003250A00EFC0BF9503250A00EFC08FF03C
:104FE000630865017370043001A07370043001A080
:104FF0000145EFC08FF96306250197B7010023AF84
:10500000875C01458545EFC09F800145EFC0EFF704
:105010006306250197B7010023A2875C03250C00D6
:10502000EFC0FF909C4089C797B7010023A8875A1B
:105030008146014681454E85EFB09FC663068500D7
:1050400097B7010023AC87588146014681455685B4
:10505000EFB0EFF46306850097B7010023A08758EF
:105060009C4089C797B7010023AA87560145EFC026
:10507000CFF16306250197B7010023A1875681462A
:10508000014681454E85EFB08FF16306850097B7E5
:10509000010023A587549C406386870097B70100D1
:1050A00023AE87520145EFC04FEE6306850097B7E8
:1050B000010023A5875281450145EFC04FF583A725
:1050C0000B008146014685078145568517B70100CB
:1050D0002322F750EFB0DFBC6306850097B70100CD
:1050E00023AE874E014597B7010023A3074EEFC0BB
:1050F000CFE909C597B7010023A2874E03250A000F
:10510000EFC0FF8203250A00EFC0CFDD6305650114
:105110007370043001A00145EFC02FE7630625013D
:1051200097B7010023AC874A03250C00EFC03F80EE
:105130009C4089C797B7010023A2874A8146014650
:1051400081454E85EFB0DFB56306850097B7010056
:1051500023A687488146014681454E85EFB02FE45E
:105160006306850097B7010023AA87469C4089C73C
:1051700097B7010023A487460145EFC00FE16306FE
:10518000250197B7010023AB87448146014681453D
:105190005685EFB0CFE06306850097B7010023AFD7
:1051A00087429C406386870097B7010023A8874207
:1051B0000145EFC08FDD09C597B7010023A08742E5
:1051C00083A70B00850717B701002325F740C9BB4C
:1051D000397152D417BA0100130A0A4022DC26DAC8
:1051E0004AD84ED656D25AD05ECE06DE62CC2A843B
:1051F000D28B094B9144954A2D49994985460146E0
:10520000DE852285EFB0AFD92285EFB05FDF85471D
:105210006306F50017B701002322F73C81460146DB
:105220002C002285EFB0DFA785476306F50017B78E
:1052300001002325F73A03270A00A2476307F70076
:10524000854717B70100232BF7382285EFB03FDBE6
:1052500011C5854717B701002322F738814601465B
:10526000DE852285EFB0AFD32285EFB05FD98547C9
:105270006306F50017B701002322F7368146014681
:105280002C002285EFB0DFA185476306F50017B734
:1052900001002325F7342285EFB07FD611C585475D
:1052A00017B70100232CF73203270A00A247630730
:1052B000F700854717B701002322F7325AC4814609
:1052C00001462C002285EFB08FCDA24785073EC452
:1052D000E3F7F4FE2285EFB09FD28D476307F50018
:1052E000854717B70100232BF72E854601462C0072
:1052F000054C228562C4EFB08FCA854601462C005A
:10530000228502C4EFB0AFC92285EFB05FCF63063C
:10531000550197B7010023A3872D854601462C0030
:105320002285EFB0CFC711C5854717B701002327E6
:10533000F72A814601462C002285EFB04FC611C5E1
:10534000854717B70100232BF72802C4854601467D
:105350006C002285EFB0DF948547814601466C00E2
:105360006306F50017B70100232AF726B247224843
:10537000228513C7F7FF6307F800854717B80100B8
:10538000232EF8243AC6EFB0BF9185476306F50097
:1053900017B701002324F724A247B246138717004A
:1053A0006388D714854797B6010023A9F6223AC42B
:1053B000E3FEE4F82285EFB09FC411C5854717B717
:1053C0000100232DF720A947814601462C002285A4
:1053D0003EC4EFB0CFBC85476306F50017B70100A8
:1053E000232EF71E814601462C0022854AC4EFB0C9
:1053F0000FBB85476306F50017B701002320F71E92
:105400002285EFB0DFBF63076501854717B701004D
:105410002326F71CA5473EC4854601462C0022855D
:10542000EFB0EFB78547630FF50A17B701002327E1
:10543000F71AA247FD173EC4E3E0F9FE2285EFB05C
:105440001FBC63075501854717B701002328F718CC
:10545000854601462C002285EFB06FB411C5854703
:1054600017B70100232CF716814601462C00228530
:10547000EFB0EFB211C5854717B701002320F7162B
:105480009D473EC4054C814601466C002285EFB025
:105490003F816306850197B7010023A18715A247C5
:1054A000B24613871700638AD70297B7010023A774
:1054B00087133AC4E379E9FC2285EFB05FB411C5E4
:1054C000854717B70100232BF71083270A008507AC
:1054D00017B701002322F71015B385073EC4E37404
:1054E000F9FAD9BFA247FD173EC4E3E7F9F2B9B70D
:1054F00085073EC4E3FCF4E475BD411126C20146B4
:10550000AA849145154506C622C4EFB02F9C97B5D5
:1055100001009385A5EF2A84EFB0FFBD2687A28600
:105520008148014881471306004097B501009385E3
:10553000E5EE170500001305E5C9EFB03FD40545BA
:10554000EFB00FD197B501009385C5ED2A84EFB078
:105550009FBAA2868148014881470147130600404F
:1055600097B50100938505ED170500001305059F0C
:10557000EFB0DFD08148014897B701009387C70497
:10558000094781461306004097B50100938505EB56
:105590001705000013058594EFB05FCEA286224464
:1055A000B24092448148014897B7010093870702AF
:1055B0000D471306004097B501009385A5E8170530
:1055C00000001305C59341016FB05FCB17B7010011
:1055D0001307870097B601009386C6FE1C439442CA
:1055E0006397F600854797B6010023A9F6FE97B7A3
:1055F0000100938727FE17B60100130666FC94434B
:1056000010426317D600854617B601002328D6FC42
:1056100097B60100938686FC18439C43884297B650
:10562000010023A1E6FA17B70100232BF7F8133581
:1056300015008280B305B500930705006386B700A7
:1056400003C70700631607003385A7406780000083
:10565000938717006FF09FFE130101FB2322910433
:10566000232C4103232291032326110423248104A4
:1056700023202105232E3103232A510323286103EC
:1056800023267103232481032320A103232EB101A8
:10569000930C0500138A05009304000063DE0500E7
:1056A0003305A0403337A000B305B040930C05008C
:1056B000338AE5409304F0FF63DA06003306C04006
:1056C000B337C000B306D040B386F640930A060055
:1056D0009389060013840C0013090A0063960628B8
:1056E00017BB0100130B0BBD6370CA16B70701008F
:1056F0006372F6149307F00F63F4C70093098000F8
:10570000B3573601330BFB0083470B001305000230
:10571000B3873701B309F540638C0900B3153A012B
:10572000B3D7FC00B31A360133E9B70033943C0118
:1057300013DB0A0193050B0013050900EF00507CF1
:10574000130A050093050B00939B0A01130509003A
:10575000EF00907693DB0B019305050013850B009A
:10576000EF00D072131A0A0193570401B367FA00CD
:1057700063FAA700B387570163E6570163F4A700F4
:10578000B38757013389A74093050B001305090020
:10579000EF001077130A050093050B0013050900AD
:1057A000EF0090711314040193050500131A0A0108
:1057B00013850B0013540401EF00506D33648A000D
:1057C000637AA40033045401636654016374A40033
:1057D000330454013304A4403354340193050000CE
:1057E000638A040033048040B3378000B305B040BF
:1057F000B385F540130504008320C104032481040C
:1058000083244104032901048329C103032A81035A
:10581000832A4103032B0103832BC102032C810242
:10582000832C4102032D0102832DC10113010105C7
:1058300067800000B707000193090001E362F6ECFE
:10584000930980016FF0DFEB631A060093050000F7
:1058500013051000EF005066930A0500B70701001A
:1058600063FAFA0E9307F00F63F45701930980006F
:10587000B3D73A01330BFB0083470B00130500023B
:1058800033095A41B3873701B309F540E38209EA86
:10589000B39A3A01335BFA00B3153A01B3D7FC006F
:1058A00093DB0A0133E9B70013050B0093850B0066
:1058B000EF001065130A050093850B00139C0A0185
:1058C00013050B00EF00505F135C0C0193050500FE
:1058D00013050C00EF00905B131A0A01935709019E
:1058E000B367FA0033943C0163FAA700B38757010A
:1058F00063E6570163F4A700B3875701338BA740D2
:1059000093850B0013050B00EF00905F130A050051
:1059100093850B0013050B00EF00105A930505004B
:1059200013050C00EF00905693160901131A0A0193
:1059300093D60601B366DA0063FAA600B386560171
:1059400063E6560163F4A600B38656013389A64088
:105950006FF01FDEB707000193090001E3EAFAF0D8
:10596000930980016FF0DFF06376DA0093050A0097
:105970006FF01FE7B707010063FAF604930BF00F0F
:1059800033B5DB001315350033D7A60097B70100F8
:1059900093874792B387E70083CB07009305000204
:1059A000B38BAB00338B7541631C0B0263E4460180
:1059B00063EACC003384CC40B306DA4033B98C00C0
:1059C00033892641930509006FF09FE1B707000175
:1059D00013050001E3EAF6FA130580016FF0DFFA20
:1059E000B3966601335D7601336DDD00B35D7A01F8
:1059F000B3156A0133DC7C0113540D01336CBC0018
:105A000013850D0093050400B3196601EF00504F94
:105A1000930A05009305040013850D0033996C016A
:105A2000931C0D01EF00504993DC0C01130A050093
:105A30009305050013850C00EF005045939A0A0169
:105A400013570C0133E7EA00930D0A00637EA700A9
:105A50003307A701930DFAFF6368A7016376A700D8
:105A6000930DEAFF3307A701330AA740930504000B
:105A700013050A00EF00D04893050400930A0500BF
:105A800013050A00EF0050439305050013040500B9
:105A900013850C00EF00903F93150C01939A0A01B7
:105AA00093D50501B3E5BA001307040063FEA50012
:105AB000B385A5011307F4FF63E8A50163F6A5000C
:105AC0001307E4FFB385A501939D0D01B70C0100F9
:105AD000B3EDED001384FCFFB3F78D0033F48900C0
:105AE000338AA54013850700930504002326F1009F
:105AF00093DD0D01EF00903993050400930A050032
:105B000013850D00EF00903813DC090193050C009C
:105B10002324A10013850D00EF0050378327C10017
:105B200013040C0093050400130C050013850700F3
:105B3000EF00D0358326810013D70A013305D50045
:105B40003307A7006374D700330C9C01B70701002B
:105B50009387F7FF935507013377F7001317070172
:105B6000B3F7FA00B3858501B307F7006366BA009F
:105B7000631EBA00637CF90033863741B3B7C700B0
:105B8000B385A541B385F54093070600B307F940F7
:105B90003339F900B305BA40B38525413394750113
:105BA000B3D767013364F400B3D565016FF05FC309
:105BB000130101FD23229102232A51012326110200
:105BC0002324810223202103232E3101232C410190
:105BD00023286101232671012324810123229101BD
:105BE0002320A101930A050093840500639E0638D3
:105BF000130406009309050017A901001309896B16
:105C000063F8C512B7070100138B05006378F6101F
:105C10001307F00F3337C70013173700B357E600E9
:105C20003309F900834609003387E6009306000232
:105C3000B386E640638C0600B394D40033D7EA0001
:105C40003314D600336B9700B399DA00935A0401EA
:105C500093850A0013050B00EF00902A1309050035
:105C600093850A00931B040113050B00EF00D02459
:105C700093DB0B01930405009305050013850B00CE
:105C8000EF00D0201319090193D70901B367F90078
:105C9000138A040063FEA700B3878700138AF4FF0A
:105CA00063E8870063F6A700138AE4FFB3878700E1
:105CB000B384A74093850A0013850400EF005024A5
:105CC0001309050093850A0013850400EF00D01E18
:105CD000939909019304050093050500131909011F
:105CE00013850B0093D90901EF00501AB3693901EC
:105CF0001386040063FCA900B30934011386F4FF82
:105D000063E6890063F4A9001386E4FF13140A0113
:105D10003364C400130A00006F000013B7070001CA
:105D200013070001E36CF6EE130780016FF01FEF1D
:105D3000138A0600631A060093050000130510007D
:105D4000EF00901713040500B7070100637EF412FB
:105D50009307F00F63F48700130A8000B3574401E0
:105D60003309F9000347090093060002330747018E
:105D7000B386E64063940612B3848440130A10008D
:105D8000135B040193050B0013850400EF0050170B
:105D90001309050093050B0013850400931B0401F0
:105DA000EF00901193DB0B019304050093050500B0
:105DB00013850B00EF00900D1319090193D709010A
:105DC000B367F900938A040063FEA700B3878700D6
:105DD000938AF4FF63E8870063F6A700938AE4FFE1
:105DE000B3878700B384A74093050B001385040095
:105DF000EF0010111309050093050B001385040033
:105E0000EF00900B93990901930405009305050099
:105E10001319090113850B0093D90901EF0010072D
:105E2000B36939011386040063FCA900B309340186
:105E30001386F4FF63E6890063F4A9001386E4FF88
:105E400013940A013364C4001305040093050A0087
:105E50008320C10203248102832441020329010219
:105E60008329C101032A8101832A4101032B0101F6
:105E7000832BC100032C8100832C4100032D0100E2
:105E80001301010367800000B7070001130A000136
:105E9000E366F4EC130A80016FF05FEC3314D40076
:105EA00033DAE400B399DA0033D7EA00935A0401F5
:105EB000B394D40093850A0013050A00336B97004E
:105EC000EF0010041309050093850A0013050A006A
:105ED000931B0401EF00407E93DB0B01930405004C
:105EE0009305050013850B00EF00407A1319090193
:105EF00013570B013367E900138A0400637EA70080
:105F000033078700138AF4FF636887006376A7006E
:105F1000138AE4FF33078700B304A74093850A0080
:105F200013850400EF00C07D1309050093850A0066
:105F300013850400EF0040789304050093050500E5
:105F400013850B00EF00807413170B011357070123
:105F500013190901B367E9001387040063FEA70062
:105F6000B38787001387F4FF63E8870063F6A70011
:105F70001387E4FFB3878700131A0A01B384A7408D
:105F8000336AEA006FF0DFDF63ECD51EB70701006C
:105F900063F4F6041307F00FB335D700939535007B
:105FA00033D7B60097A701009387C730B387E700C0
:105FB00003C70700130A00023307B700330AEA4099
:105FC00063160A0213041000E3E096E833B6CA0031
:105FD000134416006FF05FE7B70700019305000157
:105FE000E3E0F6FC930580016FF09FFBB35CE600F5
:105FF000B3964601B3ECDC0033D4E40093DB0C0130
:10600000B397440133D7EA0093850B0013050400CE
:10601000336BF700B3194601EF00806E13090500DA
:1060200093850B0013050400139C0C01EF00C0685E
:10603000135C0C01930405009305050013050C0087
:10604000EF00C0641319090113570B013367E9000E
:1060500013840400637EA700330797011384F4FFC1
:10606000636897016376A7001384E4FF3307970101
:10607000B304A74093850B0013850400EF0040682C
:106080001309050093850B0013850400EF00C0621F
:10609000930405009305050013050C00EF00005F55
:1060A00093170B011319090193D70701B367F9007F
:1060B0001386040063FEA700B38797011386F4FFDD
:1060C00063E8970163F6A7001386E4FFB38797019F
:1060D00013140401B70B01003364C4001389FBFFE0
:1060E000337D240133F92901B384A74093050900C6
:1060F00013050D00EF008059935C0401930509001E
:10610000130B050013850C00EF00405893D90901CB
:10611000130C05009385090013850C00EF00005750
:10612000130905009385090013050D00EF000056C3
:106130003305850193570B013385A70063748501EF
:106140003309790193570501B387270163E6F40208
:10615000E392F4BCB70701009387F7FF3375F500AE
:1061600013150501337BFB0033964A0133056501A6
:10617000130A0000E37AA6CC1304F4FF6FF09FB972
:10618000130A0000130400006FF01FCC130101FB81
:106190002324810423229104232E310323229103FB
:1061A0002326110423202105232C4103232A5103F4
:1061B0002328610323267103232481032320A103C1
:1061C000232EB101930C05009389050013040500EB
:1061D00093840500639E062613090600138A0600B1
:1061E00097AA0100938A0A0D63F4C514B70701004A
:1061F0006376F6129307F00F63F4C700130A80006A
:10620000B3574601B38AFA0003C70A001305000218
:1062100033074701330AE540630C0A00B39549018F
:1062200033D7EC0033194601B364B70033944C0103
:10623000935A090193850A0013850400EF00404C2E
:106240009309050093850A00131B090113850400B7
:10625000EF008046135B0B019305050013050B004F
:10626000EF00C0429399090193570401B3E7F90085
:1062700063FAA700B387270163E6270163F4A70049
:10628000B3872701B384A74093850A0013850400D0
:10629000EF0000479309050093850A001385040069
:1062A000EF0080411314040193050500939909013F
:1062B00013050B0013540401EF00403D33E4890043
:1062C000637AA40033042401636624016374A40088
:1062D000330424013304A4403355440193050000E2
:1062E0008320C1040324810483244104032901047D
:1062F0008329C103032A8103832A4103032B01035A
:10630000832BC102032C8102832C4102032D010245
:10631000832DC1011301010567800000B70700014B
:10632000130A0001E36EF6EC130A80016FF05FEDD3
:10633000631A06009305000013051000EF00C03734
:1063400013090500B7070100637AF90E9307F00FF0
:1063500063F42701130A8000B3574901B38AFA0096
:1063600003C70A0013050002B3842941330747011C
:10637000330AE540E30E0AEA33194901B3DAE900CA
:10638000B395490133D7EC0093540901336BB7003F
:1063900013850A0093850400EF00803693090500F9
:1063A00093850400931B090113850A00EF00C03098
:1063B00093DB0B019305050013850B00EF00002D07
:1063C0009399090193570B01B3E7F90033944C01FA
:1063D00063FAA700B387270163E6270163F4A700E8
:1063E000B3872701B38AA7409385040013850A0069
:1063F000EF000031930905009385040013850A001E
:10640000EF00802B9305050013850B00EF0000289B
:1064100093150B019399090193D50501B3E5B900D3
:1064200063FAA500B385250163E6250163F4A500A1
:10643000B3852501B384A5406FF09FDFB707000146
:10644000130A0001E36AF9F0130A80016FF0DFF02C
:10645000E3E8D5E8B707010063FCF604930BF00FFF
:1064600033B5DB001315350033D7A60097A701001D
:10647000938747E4B387E70083CB070093050002C7
:10648000B38BAB00338B7541631E0B0263E43601A3
:1064900063EACC003384CC40B386D94033B58C005A
:1064A000B384A64013050400938504006FF05FE3F6
:1064B000B707000113050001E3E8F6FA13058001B0
:1064C0006FF09FFAB3966601335D7601336DDD00A0
:1064D00033D47901B395690133DC7C0193540D0108
:1064E000336CBC001305040093850400B31A6601E5
:1064F000EF000021130A0500938504001305040032
:1065000033996C01931C0D01EF00001B93DC0C010F
:10651000130405009305050013850C00EF00001718
:10652000131A0A0113570C013367EA00130A040017
:10653000637EA7003307A701130AF4FF6368A7016E
:106540006376A700130AE4FF3307A701B309A74046
:106550009385040013850900EF00801A93850400D9
:106560001304050013850900EF00001593050500CD
:106570009304050013850C00EF00401193150C01E6
:106580001314040193D50501B365B4001387040007
:1065900063FEA500B385A5011387F4FF63E8A50199
:1065A00063F6A5001387E4FFB385A501131A0A015A
:1065B000B70C0100336AEA001384FCFFB3778A004A
:1065C00033F48A00B384A5401385070093050400C3
:1065D0002326F100135A0A01EF00400B930905002E
:1065E0009305040013050A00EF00400A13DC0A01BA
:1065F000930D050093050C0013050A00EF00000938
:106600008327C100130A050093050C0013850700BA
:10661000EF00C0073305B50113D709013307A70001
:106620006374B701330A9A01B70701009387F7FF34
:10663000935507013377F70013170701B3F7F900F4
:10664000B3854501B307F70063E6B400639EB40069
:10665000637CF90033865741B3B7C700B385A541C2
:10666000B385F54093070600B307F9403339F900C5
:10667000B385B440B385254133947501B3D7670121
:106680003365F400B3D565016FF09FC513060500AF
:106690001305000093F61500638406003305C5005A
:1066A00093D5150013161600E39605FE67800000CB
:1066B0006340050663C605061386050093050500BD
:1066C0001305F0FF630C060293061000637AB60010
:1066D0006358C0001316160093961600E36AB6FEC0
:1066E0001305000063E6C500B385C5403365D500DA
:1066F00093D6160013561600E39606FE6780000038
:1067000093820000EFF05FFB1385050067800200B5
:106710003305A04063D80500B305B0406FF0DFF942
:10672000B305B04093820000EFF01FF93305A0409D
:10673000678002009382000063CA0500634C050075
:10674000EFF09FF71385050067800200B305B040A6
:10675000E35805FE3305A040EFF01FF63305B040C7
:106760006780020097A70100938747E2944317A729
:106770000100130767E01843C8C2637BE50017A751
:106780000100130727E008438C4391056F905FDBFE
:10679000411122C406C617A701001307E7DE2A84A9
:1067A00008438C439105EF90BFD997A701009387C9
:1067B000E7DA9C436376F40097A7010023A087DA09
:1067C000B24022444101828097A70100938707DCF1
:1067D000984394437C43FD177CC3FC4299E3736068
:1067E00004308280011122CC26CA2A84AE844AC891
:1067F0004EC652C456C206CEEFB06FD11C4003291C
:106800000401B7090001B3E59700930AC4000CC066
:106810008144FD19370A00021840638C2A030326BD
:1068200009004A85B3654701B376360193175600D0
:10683000758F0329490063C4070001E7F1BFE39D99
:10684000E6FC9317760063D30700D58CEFC08FBBAF
:10685000E1B793C4F4FFF98C04C0EFB04FF00840E7
:10686000F2406244D2444249B249224A924A056106
:1068700082804111014506C622C4EFE01FC817E718
:10688000FFFF13074755814605469305200317A5CB
:1068900001001305E5B6EFD0EF8A19C92A84EFB0DD
:1068A0000FC82A860147814685452285EFD02F965D
:0E68B000EFB06FA0B24022440145410182804A
:02000004800278
:10000000CE44FEFFCC45FEFFD644FEFFCC45FEFFAE
:10001000CC45FEFFCC45FEFFCC45FEFFEE44FEFF87
:10002000CC45FEFFCC45FEFF0845FEFF1445FEFF14
:10003000CC45FEFF2645FEFF3245FEFF3245FEFF62
:100040003245FEFF3245FEFF3245FEFF3245FEFFE0
:100050003245FEFF3245FEFF3245FEFFCC45FEFF36
:10006000CC45FEFFCC45FEFFCC45FEFFCC45FEFF58
:10007000CC45FEFFCC45FEFFCC45FEFFCC45FEFF48
:10008000CC45FEFFCC45FEFFCC45FEFFCC45FEFF38
:10009000CC45FEFFCC45FEFFCC45FEFFCC45FEFF28
:1000A000CC45FEFFCC45FEFFCC45FEFFCC45FEFF18
:1000B000CC45FEFFCC45FEFFCC45FEFFCC45FEFF08
:1000C000CC45FEFFCC45FEFFCC45FEFFCC45FEFFF8
:1000D000CC45FEFFCC45FEFFCC45FEFFCC45FEFFE8
:1000E000CC45FEFFCC45FEFFCC45FEFFCC45FEFFD8
:1000F000CC45FEFFCC45FEFFCC45FEFFCC45FEFFC8
:100100006645FEFF7C45FEFFCC45FEFFCC45FEFF6D
:10011000CC45FEFFCC45FEFFCC45FEFFCC45FEFFA7
:10012000CC45FEFFC245FEFFCC45FEFFCC45FEFFA1
:100130007443FEFF2C44FEFFCC45FEFFCC45FEFF82
:100140006244FEFFCC45FEFFBA44FEFFCC45FEFFF5
:10015000CC45FEFFE844FEFFDA48FEFF2E49FEFFD5
:10016000E248FEFF2E49FEFF2E49FEFF2E49FEFF0C
:100170002E49FEFFD447FEFF2E49FEFF2E49FEFF0B
:10018000EE47FEFFFA47FEFF2E49FEFF0C48FEFF3A
:100190001848FEFF1848FEFF1848FEFF1848FEFFEB
:1001A0001848FEFF1848FEFF1848FEFF1848FEFFDB
:1001B0001848FEFF2E49FEFF2E49FEFF2E49FEFF86
:1001C0002E49FEFF2E49FEFF2E49FEFF2E49FEFF5F
:1001D0002E49FEFF2E49FEFF2E49FEFF2E49FEFF4F
:1001E0002E49FEFF2E49FEFF2E49FEFF2E49FEFF3F
:1001F0002E49FEFF2E49FEFF2E49FEFF2E49FEFF2F
:100200002E49FEFF2E49FEFF2E49FEFF2E49FEFF1E
:100210002E49FEFF2E49FEFF2E49FEFF2E49FEFF0E
:100220002E49FEFF2E49FEFF2E49FEFF2E49FEFFFE
:100230002E49FEFF2E49FEFF2E49FEFF2E49FEFFEE
:100240002E49FEFF2E49FEFF2E49FEFF2E49FEFFDE
:100250002E49FEFF2E49FEFF4C48FEFF7A48FEFF66
:100260002E49FEFF2E49FEFF2E49FEFF2E49FEFFBE
:100270002E49FEFF2E49FEFF2E49FEFFD048FEFF0D
:100280002E49FEFF2E49FEFF3246FEFF2C47FEFFA1
:100290002E49FEFF2E49FEFF9E47FEFF2E49FEFF20
:1002A000C447FEFF2E49FEFF2E49FEFF2849FEFFF0
:1002B000000102020303030304040404040404040D
:1002C00005050505050505050505050505050505DE
:1002D00006060606060606060606060606060606BE
:1002E00006060606060606060606060606060606AE
:1002F000070707070707070707070707070707078E
:10030000070707070707070707070707070707077D
:10031000070707070707070707070707070707076D
:10032000070707070707070707070707070707075D
:10033000080808080808080808080808080808083D
:10034000080808080808080808080808080808082D
:10035000080808080808080808080808080808081D
:10036000080808080808080808080808080808080D
:1003700008080808080808080808080808080808FD
:1003800008080808080808080808080808080808ED
:1003900008080808080808080808080808080808DD
:1003A00008080808080808080808080808080808CD
:1003B000546D725100000000546D7220537663003A
:1003C000286E756C6C2900004572726F7220696E20
:1003D0002047656E5154657374207461736B73208C
:1003E0000D0A00006D69616F750A00006D69616F2B
:1003F00075320A0068756E6772790A004368656332
:100400006B54696D6572000047656E5F5175657567
:10041000655F54657374000047656E51000000000D
:1004200047656E5F51756575655F4D7574657800DC
:100430004D754C6F770000004D754D6564000000F0
:080440004D7548696768000072
:100448001000000000000000017A5200017C010148
:100458001B0D02005000000018000000F451FEFFC0
:100468005805000000440E507489039406990B81C6
:1004780001880292049305950796089709980A9AA5
:100488000C9B0D036C010AC144C844C944D244D32F
:1004980044D444D544D644D744D844D944DA44DB78
:1004A800440E00440B0000004C0000006C000000EB
:1004B800F856FEFFDC05000000440E3070890395F5
:1004C8000781018802920493059406960897099873
:1004D8000A990B9A0C0370020AC144C844C944D251
:1004E80044D344D444D544D644D744D844D944DA30
:1004F800440E00440B00000050000000BC00000047
:10050800845CFEFF0005000000440E5074880289D8
:10051800039305990B810192049406950796089711
:1005280009980A9A0C9B0D0320010AC144C844C9C2
:1005380044D244D344D444D544D644D744D844D9E7
:0C05480044DA44DB440E00440B000000C9
:0805DC00FC8F01000900000082
:040000058000004037
:00000001FF
